:040000007FEF2DF071
:1000080000C076F001C015F0E1CF77F0E2CF78F0CC
:10001800F2A808D0F2A206D0010E0901FE6F000E68
:10002800FF6FF2929DAA67D09EAA65D0AECF8BFAD9
:10003800ABA20FD0AB98AECF8BFAAB88010E0B01F9
:100048006A25006E000E6B21016E00C06AFB01C0BC
:100058006BFBABA40FD00B01AB9EAB8E010E6A25D8
:10006800006E000E6B21016E00C06AFB01C06BFBC5
:10007800AECF8BFA0A018B510D0A07E08F510008A9
:1000880002E18E51500801E320D0010E8C6F000E62
:100098008D6F8F51000802E18E51500804E2020E64
:1000A8008C6F000E8D6F9D9A920E8E25E16E0A0E52
:1000B8008F21E26EE66A8ECA90FA8FCA91FA9D9AEB
:1000C800F2928E6B8F6B8B6B16D0920E8E25E16E33
:1000D8000A0E8F21E26E8BCAE6FF8ECA90FA8FCA8B
:1000E80091FA010E8E25006E000E8F21016E00C060
:1000F8008EFA01C08FFA9DA01ED09EA01CD0010EC2
:100108000B016E5D006E000E6F59016E00C06EFB34
:1001180001C06FFB000E6F5D02E1010E6E5D06E22D
:100128009D90CD90010E6C6F000E6D6F3C0ECF6EE2
:10013800B00ECE6E9E9076C000F015C001F077C06C
:08014800E1FF78C0E2FF1100A5
:100150000B820BAEB2EF00F0036802680168006822
:080160000A360232FF0E120004
:0E016800026A016A006A086A036A000E120049
:100176000B840BAEC6EF00F0010E036E026A016A35
:0A018600006A0A360232FF0E120072
:080190000AAE029E000E1200EF
:100198000CB00EEF01F00CA2B4EF01F00E6A000EE5
:1001A800026425EF01F0F00E0214D8A4F0EF00F07D
:1001B800023A01380F0B02260138F00B016E0038A5
:1001C8000F0B01260038F00B006E08380F0B0026C5
:1001D8000838F00B086E0E84D89002BE09EF01F0C3
:1001E80008360036013602360E2A02BE09EF01F043
:1001F80008360036013602360E2A02BE09EF01F033
:1002080008360036013602360E2A0E500364AAEF6D
:1002180001F0035E0BBC08AEAFEF01F0D880800E92
:1002280008640030000E002201220222D8A0AFEF9D
:1002380001F0023201320032034AB4EF01F0AFEFAD
:1002480001F001C002F000C001F008C000F0086A27
:10025800000E0E8602645CEF01F0F00E0214D8A4C2
:1002680044EF01F0023A01380F0B02260138F00B77
:10027800016E00380F0B01260038F00B006E0E845B
:10028800D89002BE09EF01F00036013602360E2A78
:1002980002BE09EF01F00036013602360E2A02BE10
:1002A80009EF01F00036013602360E2A09EF01F097
:1002B80001C002F000C001F0006A000E0E960E8820
:1002C800026489EF01F0F00E0214D8A474EF01F073
:1002D800023A01380F0B02260138F00B016E0E842A
:1002E800D89002BE09EF01F0013602360E2A02BE8E
:1002F80009EF01F0013602360E2A02BE09EF01F0BD
:10030800013602360E2A09EF01F001C002F0016A37
:10031800000E0E860264B9EF01F0F00E0214D8A4A4
:1003280098EF01F0023A0E84D89002BE09EF01F06E
:1003380002360E2A02BE09EF01F002360E2A02BE6C
:1003480009EF01F002360E2A09EF01F0010E0C6EDA
:100358000EDFBCEF01F0020E0C6E16DFBCEF01F0F1
:10036800040E0C6EF1DEBCEF01F0080E0C6EF8DE28
:02037800120071
:0E037A00ACB202D00000FCD7B7CBADFF120032
:0C03880072B201D0FDD7B7CB73FF12009A
:100394000134083609360450085E0550D8A0053CDF
:1003A400095E003601360F0E0C6E0134083609362C
:1003B400045000A006D0085E0550D8A0053C095E94
:1003C40005D008260550D8B0053C0926003601366C
:1003D4000C2EEBD700B006D0045008260550D8B038
:0803E400053C0926000012008F
:1003EC00025006180E6E086A096A0B6A03500764FD
:1003FC00E9EF02F006500A6E068E028E03500B6E69
:10040C000750036E000E0B6439EF02F00B50075EC1
:10041C00D8B4DAEF02F0070E0764A8EF02F0075E1B
:10042C0000C008F001C000F002C001F0026A074EE3
:10043C00DAEF02F007647DEF02F0075E00C008F00F
:10044C0001C000F0016A074EDAEF02F007645BEFBF
:10045C0002F0075E00C008F0006A074EDAEF02F007
:10046C00076442EF02F00AC002F005C001F004C0BC
:10047C0000F0086A03EF04F0030E07644DEF02F07E
:10048C00075E08380F0B086E074EDAEF02F0D890B3
:10049C000832074EDAEF02F0D8900832074EDAEF46
:1004AC0002F0D8900832DAEF02F0030E07646CEF1A
:1004BC0002F0075E08380F0B086E0038F00B0826A8
:1004CC0000380F0B006E074EDAEF02F0D8900032B6
:1004DC000832074EDAEF02F0D89000320832074E9D
:1004EC00DAEF02F0D89000320832DAEF02F0030EA5
:1004FC00076494EF02F0075E08380F0B086E0038A3
:10050C00F00B082600380F0B006E0138F00B00269C
:10051C0001380F0B016E074EDAEF02F0D890013262
:10052C0000320832074EDAEF02F0D8900132003276
:10053C000832074EDAEF02F0D8900132003208325E
:10054C00DAEF02F0030E0764C5EF02F0075E08381D
:10055C000F0B086E0038F00B082600380F0B006EDE
:10056C000138F00B002601380F0B016E0238F00B2E
:10057C00012602380F0B026E074EDAEF02F0D8900C
:10058C000232013200320832074EDAEF02F0D89014
:10059C000232013200320832074EDAEF02F0D89004
:1005AC000232013200320832096A000E0EAECEEF72
:1005BC0003F0081E001E011E021E082A0022012242
:1005CC000222CEEF03F00750D8A4EFEF02F003EFB6
:1005DC0004F0096A02C00AF0028E068E0750035C12
:1005EC00076ED8B4C1EF03F0070E07648FEF03F06A
:1005FC00075E0450096E0550046E0650056E066ABF
:10060C00074EC1EF03F0070E076464EF03F0075EBB
:10061C000450096E0550046E056A074EC1EF03F0D5
:10062C00070E076442EF03F0075E0450096E046A7C
:10063C00074EC1EF03F0070E076429EF03F00AC061
:10064C0002F003EF04F0030E076434EF03F0075ECF
:10065C0009380F0B096E074EC1EF03F0D890093221
:10066C00074EC1EF03F0D8900932074EC1EF03F0EB
:10067C00D8900932C1EF03F0030E076453EF03F077
:10068C00075E09380F0B096E0438F00B0926043885
:10069C000F0B046E074EC1EF03F0D89004320932F1
:1006AC00074EC1EF03F0D89004320932074EC1EF68
:1006BC0003F0D89004320932C1EF03F0030E076443
:1006CC007BEF03F0075E09380F0B096E0438F00B53
:1006DC00092604380F0B046E0538F00B0426053878
:1006EC000F0B056E074EC1EF03F0D89005320432A4
:1006FC000932074EC1EF03F0D890053204320932AB
:10070C00074EC1EF03F0D890053204320932C1EF25
:10071C0003F0030E0764ACEF03F0075E09380F0B10
:10072C00096E0438F00B092604380F0B046E0538DB
:10073C00F00B042605380F0B056E0638F00B05265A
:10074C0006380F0B066E074EC1EF03F0D890063239
:10075C00053204320932074EC1EF03F0D89006324D
:10076C00053204320932074EC1EF03F0D89006323D
:10077C00053204320932086A000E0EAECEEF03F0D9
:10078C00091E041E051E061E092A04220522062225
:10079C00095008260450002205500122065002225E
:1007AC000EBEE5EF03F0D8A0F4EF03F002320132F5
:1007BC0000320832033EF4EF03F0FEEF03F0D8B042
:1007CC00F9EF03F0000E081E001E011E021E082A7F
:1007DC000022012202220A7EF9EF03F0010E0C6EB8
:1007EC00D5DC05EF04F0020E0C6ED0DC05EF04F046
:1007FC00040E0C6EA7DC05EF04F0000E0C6E12005C
:10080C00086A096A000E076203648BEF04F0025059
:10081C0006180A6E075003267E0ED8A01CEF04F0B3
:10082C00035ED8B08FEF04F020EF04F0035ED8A085
:10083C0093EF04F0028E068E02C00EF001C00BF096
:10084C0000C00DF000500402F4CF0CF00150050272
:10085C00F4CF00F0F3CF08F00402F3500C26F45060
:10086C000822000E00220D500502F3500C26F45005
:10087C000822000E002202500402F3500826F45005
:10088C00002202500502016A000E0122F3500026DC
:10089C00F45001220D500602F3500826F4500022A9
:1008AC00026A000E012202220B500602F3500026AF
:1008BC00F4500122000E02220E500602F3500126C3
:1008CC00F450022202BE73EF04F0083600360136F3
:1008DC0002360306D8B493EF04F086EF04F0D88008
:1008EC00800E08640030000E002201220222D8A0E3
:1008FC0086EF04F0023201320032034A8FEF04F02B
:10090C000AAE029E000E95EF04F0010E27DC95EF67
:10091C0004F0020E17DC95EF04F0040E26DC120036
:10092C000D6A086A0050D8B4000C04180A6E0ABE8E
:10093C000D1E0B6A04AE02D0041E042A00AE02D0B7
:10094C00001E002A005004100A6E0ABE1FD004506C
:10095C00085E003600340836045008260036060EB1
:10096C000C6E00340836045000B0085E00A0082657
:10097C0000360C2EF6D700A008260BB015D00DAE05
:10098C00000C001E002A081E082A000C04AE09D018
:10099C0000BE04D00050086E006AF1D7006A002A2D
:1009AC00000C001E0B2AD3D7082A0450085CD8A4CC
:0E09BC00E6D7086A002A00AEE2D7FF0C120050
:1009CA000B800BAEF1EF04F0026A0AAEFF0E026E64
:0C09DA00016E006E0A360232FF0E1200A1
:0809E6000B6A0B86FF0E1200E4
:1009EE00B6CB04F08B92026A036A800E0318006E77
:1009FE00800E005C02E1080E025C1FE2800E041401
:100A0E00016E0150800A02E18B8201D08B922A0E78
:100A1E000D6E0D2EFED70000043604908B842A0E28
:100A2E000D6E0D2EFED700008B942A0E0D6E0D2E20
:0C0A3E00FED70000024A032AD8D712009D
:100A4A00086A080E0C6E003408360450085ED8B0E6
:0E0A5A0002D00826D89000360C2EF5D71200D8
:100A6800C7B409D01F0EC514016E0150000A03E176
:0A0A7800010E006E01D0006A1200AA
:100A8200F250026EF29E0500FF6A0150FE6E0050A7
:080A9200FD6E02BEF28E12009F
:100A9A000050086E0150006E0250016E0350026E43
:100AAA00036A0B6A0C6A9E0E036E0A6A020E0C6EC9
:060ABA00CCEC00F012007C
:100AC0000B6A0C6A086A0350D8B4E4EF05F002C060
:100AD0000AF0028E9E0E035E03AED4EF05F0036CA7
:100AE000080E035CD8A0A1EF05F0036E083600C025
:100AF00008F001C000F002C001F0026A080E035CB9
:100B0000D8A0A1EF05F0036E083600C008F001C0C0
:100B100000F0016A080E035CD8A0A1EF05F0036E97
:100B2000083600C008F0006A080E035CD8A0A1EFE8
:100B300005F0036E0836086A0350D8A4D890ADEFCC
:100B400005F00350D8B4ADEF05F0D8900232013271
:100B500000320832032EA5EF05F00BBC08A0BEEF53
:100B600005F0D8A0BEEF05F0082AD8B4002AD8B402
:100B7000012AD8B4022A02BEE8EF05F00AAEE4EF7B
:100B800005F0021E011E001E081E082AD8B4002A05
:100B9000D8B4012AD8B4022AE4EF05F0026A016A47
:100BA000006A086AE4EF05F00B800BAEEEEF05F08B
:100BB000026A0AAEEEEF05F0026E016E006E086E7C
:100BC0000A360232EEEF05F00C6A000EEFEF05F088
:100BD000010E0C6E000EF9DEEFEF05F0FF0E025075
:100BE000036E0150026E0050016E0850006E12003C
:080BF000067EF6EC01F0120094
:100BF8008B900A0E0D6E0D2EFED70000A9CBB6FB0A
:100C0800F2DEB2CBB6FBEFDEA9CBB6FBECDEB3CBA4
:100C1800B6FBE9DEA9CBB6FBE6DEB4CBB6FBE3DE7A
:100C2800A9CBB6FBE0DEB5CBB6FBDDDEA9CBB6FBC8
:100C3800DADEB1CBB6FBD7DEA9CBB6FBD4DEB0CBC0
:100C4800B6FBD1DEA9CBB6FBCEDEAFCBB6FBCBDE97
:100C5800A9CBB6FBC8DEAECBB6FBC5DEA9CBB6FBCF
:100C6800C2DEADCBB6FBBFDEA9CBB6FBBCDEACCBE0
:100C7800B6FBB9DEA9CBB6FBB6DEABCBB6FBB3DEB3
:100C8800A9CBB6FBB0DEAACBB6FBADDE0A0E0D6E65
:100C98000D2EFED700008B800A0E0D6E0D2EFED78E
:040CA8000000120036
:100CAC000B6A0A6A096A086A0E6A03340836045029
:100CBC00085E0550D8A0053C095E0650D8A0063C3D
:100CCC000A5E0750D8A0073C0B5EE86AD8A0010E5C
:100CDC000E5E0336070E0C6E0334083609360A36E0
:100CEC000B360E36045003A012D0085E0550D8A067
:100CFC00053C095E0650D8A0063C0A5E0750D8A0F9
:100D0C00073C0B5EE86AD8A0010E0E5E11D00826D7
:100D1C000550D8B0053C09260650D8B0063C0A262A
:100D2C000750D8B0073C0B26E86AD8B0010E0E2647
:100D3C0003360C2ED1D70234083609360A360B3658
:100D4C000E36045003A012D0085E0550D8A0053C06
:100D5C00095E0650D8A0063C0A5E0750D8A0073C96
:100D6C000B5EE86AD8A0010E0E5E11D00826055065
:100D7C00D8B0053C09260650D8B0063C0A260750C8
:100D8C00D8B0073C0B26E86AD8B0010E0E26023606
:100D9C00070E0C6E0234083609360A360B360E3640
:100DAC00045002A012D0085E0550D8A0053C095E84
:100DBC000650D8A0063C0A5E0750D8A0073C0B5E34
:100DCC00E86AD8A0010E0E5E11D008260550D8B0E6
:100DDC00053C09260650D8B0063C0A260750D8B068
:100DEC00073C0B26E86AD8B0010E0E2602360C2EF4
:100DFC00D1D70134083609360A360B360E36045074
:100E0C0002A012D0085E0550D8A0053C095E065021
:100E1C00D8A0063C0A5E0750D8A0073C0B5EE86AD7
:100E2C00D8A0010E0E5E11D008260550D8B0053C96
:100E3C0009260650D8B0063C0A260750D8B0073C05
:100E4C000B26E86AD8B0010E0E260136070E0C6E82
:100E5C000134083609360A360B360E36045001A01A
:100E6C0012D0085E0550D8A0053C095E0650D8A0EB
:100E7C00063C0A5E0750D8A0073C0B5EE86AD8A077
:100E8C00010E0E5E11D008260550D8B0053C09267F
:100E9C000650D8B0063C0A260750D8B0073C0B26A3
:100EAC00E86AD8B0010E0E2601360C2ED1D70034CC
:100EBC00083609360A360B360E36045001A012D00D
:100ECC00085E0550D8A0053C095E0650D8A0063C2B
:100EDC000A5E0750D8A0073C0B5EE86AD8A0010E4A
:100EEC000E5E11D008260550D8B0053C09260650D8
:100EFC00D8B0063C0A260750D8B0073C0B26E86A47
:100F0C00D8B0010E0E260036070E0C6E00340836D3
:100F1C0009360A360B360E36045000A012D0085E85
:100F2C000550D8A0053C095E0650D8A0063C0A5EC8
:100F3C000750D8A0073C0B5EE86AD8A0010E0E5EE5
:100F4C0011D008260550D8B0053C09260650D8B05B
:100F5C00063C0A260750D8B0073C0B26E86AD8B0E6
:100F6C00010E0E2600360C2ED1D700B00ED0045038
:100F7C0008260550D8B0053C09260650D8B0063CCA
:0C0F8C000A260750D8B0073C0B261200C4
:100F98006E0E0B01A95DD8A0C6D0640E046EA9CB55
:100FA80000F04FDD120E0024056E066A000E0622C0
:100FB80005C000F006C001F0000E06BEFF0E026E6E
:100FC800036E003600900136023603360036009074
:100FD8000136023603364D0E0024F66E7F0E0120D0
:100FE800F76E000E0220F86E0900F5CF00F0090038
:100FF800F5CF01F00900F5CF02F00900F5CF03F0B5
:10100800000E046E000E056E000E066E7E0E076E54
:1010180006EC04F000C0AAFB01C0ABFB02C0ACFBAD
:1010280003C0ADFB640E046EA9CB00F00ADD08C056
:1010380000F00A0E046E05DD090E0024056E066A2E
:10104800000E062205C000F006C001F0000E06BE24
:10105800FF0E026E036E003600900136023603362C
:10106800003600900136023603364D0E0024F66E27
:101078007F0E0120F76E000E0220F86E0900F5CFF2
:1010880000F00900F5CF01F00900F5CF02F00900E2
:10109800F5CF03F0AACB04F0ABCB05F0ACCB06F050
:1010A800ADCB07F006EC04F000C0AAFB01C0ABFB17
:1010B80002C0ACFB03C0ADFB0A0E046EA9CB00F066
:1010C800C0DC08C000F000C001F0000E026E036E24
:1010D800046E01360190023603360436013601905B
:1010E8000236033604364D0E0124F66E7F0E0220BA
:1010F800F76E000E0320F86E0900F5CF00F0090026
:10110800F5CF01F00900F5CF02F00900F5CF03F0A3
:10111800AACB04F0ABCB05F0ACCB06F0ADCB07F017
:1011280006EC04F0AFD0A9510A08D8B07CD00A0E5A
:10113800046EA9CB00F085DC090E0024056E066A52
:10114800000E062205C000F006C001F0000E06BE23
:10115800FF0E026E036E003600900136023603362B
:10116800003600900136023603364D0E0024F66E26
:101178007F0E0120F76E000E0220F86E0900F5CFF1
:1011880000F00900F5CF01F00900F5CF02F00900E1
:10119800F5CF03F0000E046E000E056E000E066E0D
:1011A8007E0E076E06EC04F000C0AAFB01C0ABFB84
:1011B80002C0ACFB03C0ADFB0A0E046EA9CB00F065
:1011C80040DC08C000F000C001F0000E026E036EA3
:1011D800046E01360190023603360436013601905A
:1011E8000236033604364D0E0124F66E7F0E0220B9
:1011F800F76E000E0320F86E0900F5CF00F0090025
:10120800F5CF01F00900F5CF02F00900F5CF03F0A2
:10121800AACB04F0ABCB05F0ACCB06F0ADCB07F016
:1012280006EC04F02FD0A9CB00F0000E016E026E80
:10123800036E003600900136023603360036009001
:101248000136023603364D0E0024F66E7F0E01205D
:10125800F76E000E0220F86E0900F5CF00F00900C5
:10126800F5CF01F00900F5CF02F00900F5CF03F042
:10127800000E046E000E056E000E066E7E0E076EE2
:0612880006EC04F0120068
:10128E0007C1A9FB08C1AAFB09C1ABFB0AC1ACFB94
:10129E00C582C5A221D001010751081109110A11F9
:1012AE001AE00B01A951AA11AB11AC110DE1EBC95A
:1012BE00E1FFECC9E2FF060EE66EE9C900F0EAC9ED
:1012CE0001F041EC05F008D0010E0B01A95F000EF4
:0A12DE00AA5BAB5BAC5BDDD712002E
:1012E8000A6A0350D8A40A800750D8A40A820A5070
:1012F800D8B4D7EF09F0030AD8B490EF09F00AB0D0
:101308008BEF09F006AED5EF09F0D3EF09F002AE86
:10131800D3EF09F0D5EF09F00250800B0A6E029E58
:101328000650800B069E0A18D8B4A1EF09F00A509F
:10133800D8B4D3EF09F0D5EF09F00750035CD8B45F
:10134800ABEF09F0D8A0C7EF09F0CDEF09F00650D0
:10135800025CD8B4B5EF09F0D8A0C7EF09F0CDEF1B
:1013680009F00550015CD8B4BFEF09F0D8A0C7EF69
:1013780009F0CDEF09F00450005CD8B4D7EF09F0BC
:10138800D8B0CDEF09F00A52D8B4D5EF09F0D3EFB1
:1013980009F00A52D8B4D3EF09F0D5EF09F0D88094
:0E13A8001200D8901200D880D88412001200D3
:1013B60003500718D8A4EFEF09F002500618D8A476
:1013C600EFEF09F001500518D8A4EFEF09F000502F
:0E13D6000418D8B4D8841200D8941200120063
:1013E4000B01A951390806E3300EA95D03E3010E90
:0813F400006E01D0006A120036
:1013FC000B6A0A6A096A00500402F4CF09F0F3CFB1
:10140C0008F001500502F4CF0BF0F3CF0AF00050B6
:10141C000502F3500926F4500A22E86A0B22015007
:10142C000402F3500926F4500A22E86A0B2208C081
:10143C0000F009C001F00AC002F00BC003F012006A
:10144C0007C1ABFB08C1ACFB09C1ADFB0AC1AEFBCC
:10145C009E96C5869EB621D001010751081109112F
:10146C000A111AE00B01AB51AC11AD11AE110DE12B
:10147C00EBC9E1FFECC9E2FF030EE66EE9C900F02F
:10148C00EAC901F041EC05F008D0010E0B01AB5F8D
:10149C00000EAC5BAD5BAE5BDDD70B01C9CFAAFB1D
:1014AC00A951000A02E1C58A01D0C59A9E96C58849
:1014BC0007C1ABFB08C1ACFB09C1ADFB0AC1AEFB5C
:1014CC009EB621D001010751081109110A111AE029
:1014DC000B01AB51AC11AD11AE110DE1EBC9E1FF3C
:1014EC00ECC9E2FF030EE66EE9C900F0EAC901F0AF
:1014FC0041EC05F008D0010E0B01AB5F000EAC5BAC
:0C150C00AD5BAE5BDDD7AACB00F0120097
:101518000450000A08E10550000A05E1FF0E006EBC
:101528007F0E016E58D00D6A096A086A01500010D2
:10153800D8B4000C015005180A6E0ABE0D1E0B6ABD
:1015480005AE05D0041E051E042AD8B4052A01AE2E
:1015580005D0001E011E002AD8B4012A015005102A
:101568000A6E0ABE10D0CAEC01F00BB020D00DAE46
:10157800000C001E011E002AD8B4012A081E091EEC
:10158800082AD8B4092A000C05AE0DD001BE07D030
:101598000150096E0050086E016A006AE8D7016AB6
:1015A800006A002A000C011E001E0B2ADDD7082A3B
:1015B800D8B4092A0450085CD8A4D9D70550095CC6
:1015C800D8A4D5D7096A086A002AD8B4012A01AE76
:0815D800CED70000FF0C120049
:1015E000800E0B01A919006E800E000A005CD8B0B5
:1015F0006DD1A9510008016E01C0A9FB800E011830
:10160000006E800E6E0A005CD8A0C0D0640E046E1E
:10161000A9CB00F096EC04F0120E0024056E000E2B
:1016200000BEFF0E066E000E062205C000F006C0CA
:1016300001F0000E06BEFF0E026E036E0036009033
:101640000136023603360036009001360236033684
:101650004D0E0024F66E7F0E0120F76E000E022064
:10166000F86E0900F5CFAAFB0900F5CFABFB090026
:10167000F5CFACFB0900F5CFADFB640E046EA9CB32
:1016800000F096EC04F008C000F00A0E046E96EC30
:1016900004F0090E0024056E000E00BEFF0E066E5B
:1016A000000E062205C000F006C001F0000E06BEC6
:1016B000FF0E026E036E00360090013602360336CE
:1016C000003600900136023603364D0E0024F66EC9
:1016D0007F0E0120F76E000E0220F86E0900F5CF94
:1016E00000F00900F5CF01F00900F5CF02F0090084
:1016F000F5CF03F0AACB04F0ABCB05F0ACCB06F0F2
:10170000ADCB07F006EC04F000C0AAFB01C0ABFBB8
:1017100002C0ACFB03C0ADFB0A0E046EA9CB00F007
:1017200096EC04F008C000F000C001F0000E00BE0E
:10173000FF0E026E036E046E013601900236033610
:101740000436013601900236033604364D0E01246C
:10175000F66E7F0E0220F76E000E0320F86E090071
:10176000F5CF00F00900F5CF01F00900F5CF02F048
:101770000900F5CF03F0AACB04F0ABCB05F0ACCB5E
:1017800006F0ADCB07F006EC04F007D2800E0A0A93
:10179000006E800EA919005C71E20A0E046EA9CBDE
:1017A00000F096EC04F0090E0024056E000E00BE59
:1017B000FF0E066E000E062205C000F006C001F006
:1017C000000E06BEFF0E026E036E0036009001365C
:1017D00002360336003600900136023603364D0ECF
:1017E0000024F66E7F0E0120F76E000E0220F86EC8
:1017F0000900F5CFAAFB0900F5CFABFB0900F5CF37
:10180000ACFB0900F5CFADFB0A0E046EA9CB00F0CE
:1018100096EC04F008C000F000C001F0000E00BE1D
:10182000FF0E026E036E046E01360190023603361F
:101830000436013601900236033604364D0E01247B
:10184000F66E7F0E0220F76E000E0320F86E090080
:10185000F5CF00F00900F5CF01F00900F5CF02F057
:101860000900F5CF03F0AACB04F0ABCB05F0ACCB6D
:1018700006F0ADCB07F006EC04F08FD1A9CB00F059
:10188000000EA9BFFF0E016E026E036E00360090BF
:101890000136023603360036009001360236033632
:1018A0004D0E0024F66E7F0E0120F76E000E022012
:1018B000F86E0900F5CF00F00900F5CF01F009003E
:1018C000F5CF02F00900F5CF03F067D1800EA9191A
:1018D000006E800E6E0A005CD8A0C0D0640E046E4C
:1018E000A9CB00F096EC04F0120E0024056E000E59
:1018F00000BEFF0E066E000E062205C000F006C0F8
:1019000001F0000E06BEFF0E026E036E0036009060
:1019100001360236033600360090013602360336B1
:10192000810E0024F66E7F0E0120F76E000E02205D
:10193000F86E0900F5CFAAFB0900F5CFABFB090053
:10194000F5CFACFB0900F5CFADFB640E046EA9CB5F
:1019500000F096EC04F008C000F00A0E046E96EC5D
:1019600004F0090E0024056E000E00BEFF0E066E88
:10197000000E062205C000F006C001F0000E06BEF3
:10198000FF0E026E036E00360090013602360336FB
:1019900000360090013602360336810E0024F66EC2
:1019A0007F0E0120F76E000E0220F86E0900F5CFC1
:1019B00000F00900F5CF01F00900F5CF02F00900B1
:1019C000F5CF03F0AACB04F0ABCB05F0ACCB06F01F
:1019D000ADCB07F006EC04F000C0AAFB01C0ABFBE6
:1019E00002C0ACFB03C0ADFB0A0E046EA9CB00F035
:1019F00096EC04F008C000F000C001F0000E00BE3C
:101A0000FF0E026E036E046E01360190023603363D
:101A1000043601360190023603360436810E012465
:101A2000F66E7F0E0220F76E000E0320F86E09009E
:101A3000F5CF00F00900F5CF01F00900F5CF02F075
:101A40000900F5CF03F0AACB04F0ABCB05F0ACCB8B
:101A500006F0ADCB07F006EC04F09FD0800E0A0A2A
:101A6000006E800EA919005C71E20A0E046EA9CB0B
:101A700000F096EC04F0090E0024056E000E00BE86
:101A8000FF0E066E000E062205C000F006C001F033
:101A9000000E06BEFF0E026E036E00360090013689
:101AA0000236033600360090013602360336810EC8
:101AB0000024F66E7F0E0120F76E000E0220F86EF5
:101AC0000900F5CFAAFB0900F5CFABFB0900F5CF64
:101AD000ACFB0900F5CFADFB0A0E046EA9CB00F0FC
:101AE00096EC04F008C000F000C001F0000E00BE4B
:101AF000FF0E026E036E046E01360190023603364D
:101B0000043601360190023603360436810E012474
:101B1000F66E7F0E0220F76E000E0320F86E0900AD
:101B2000F5CF00F00900F5CF01F00900F5CF02F084
:101B30000900F5CF03F0AACB04F0ABCB05F0ACCB9A
:101B400006F0ADCB07F006EC04F027D0A9CB00F0EF
:101B5000000EA9BFFF0E016E026E036E00360090EC
:101B6000013602360336003600900136023603365F
:101B7000810E0024F66E7F0E0120F76E000E02200B
:101B8000F86E0900F5CF00F00900F5CF01F009006B
:0C1B9000F5CF02F00900F5CF03F01200C1
:101B9C000450000A12E10550000A0FE10650000A39
:101BAC000CE10750000A09E1FF0E006EFF0E016EFA
:101BBC007F0E026EFF0E036EA8D0086A096A0750EA
:101BCC00D8B479EF0EF00350D8B47EEF0EF002507B
:101BDC0006180A6E028E068E0E6A02C008F001C04C
:101BEC000CF000C00DF004500D5E0550D8A0053C63
:101BFC000C5E0650D8A0063C085E086A0C6A0D6A9A
:101C0C00D8A010EF0EF0D890023201320032083218
:101C1C00010E0E6E0750035ED8A01DEF0EF07E0E67
:101C2C000E240326D8B083EF0EF023EF0EF07E0EB9
:101C3C000E240326D8A088EF0EF0180E0B6E0D366E
:101C4C000C3608360036013602360E360450005E6D
:101C5C000550D8A0053C015E0650D8A0063C025E9B
:101C6C0006340E120EA03EEF0EF00D8049EF0EF072
:101C7C00045000260550D8B0053C01260650D8B0BB
:101C8C00062802260D900B2E25EF0EF06FEF0EF0AE
:101C9C00D8900036013602360E360450005E0550E0
:101CAC00D8A0053C015E0650D8A0063C025E063466
:101CBC000E10010B0D26D8B00C2AD8B4082AD8A4C3
:101CCC006FEF0EF008320C320D32032AD8B483EFCA
:101CDC000EF00AAE089E0850026E0C50016E0D50AC
:101CEC00006E8BEF0EF0010EF3EC04F08BEF0EF0A8
:101CFC00020EB4EC00F08BEF0EF0040EA8EC00F02A
:0C1D0C008BEF0EF0080EBBEC00F0120094
:101D18000B6A0C6A0A6A086A0350D8B414EF0FF009
:101D2800028E9E0E035E03BE9FEF0EF0D8B49FEFA7
:101D38000EF004EF0FF0036C080E035CD8A0D1EF8F
:101D48000EF0036E083600C008F001C000F002C0B3
:101D580001F0026A080E035CD8A0D1EF0EF0036E02
:101D6800083600C008F001C000F0016A080E035CE4
:101D7800D8A0D1EF0EF0036E083600C008F0006A54
:101D8800080E035CD8A0D1EF0EF0036E0836086A7F
:101D98000350D8A4D890DDEF0EF00350D8B4DDEF8F
:101DA8000EF0D8900232013200320832032ED5EFFD
:101DB8000EF00BBC08A0EEEF0EF0D8A0EEEF0EF080
:101DC800082AD8B4002AD8B4012AD8B4022A02BEF4
:101DD80018EF0FF00AAE14EF0FF0021E011E001EDE
:101DE800081E082AD8B4002AD8B4012AD8B4022A6E
:101DF80014EF0FF0026A016A006A086A14EF0FF024
:101E08000B800BAE1EEF0FF0026A0AAE1EEF0FF04A
:101E1800026E016E006E086E0A3602321EEF0FF077
:101E2800000E0C6A1FEF0FF0010E0C6EE5EC04F0CB
:101E38001FEF0FF0FF0E0250036E0150026E0050AC
:081E4800016E0850006E12004B
:041E5000C584120033
:101E54009E96A9CBC9FF07C1AAFB08C1ABFB09C168
:101E6400ACFB0AC1ADFBC7A423D001010751081183
:101E740009110A111CE00B01AA51AB11AC11AD11EF
:101E84000FE1EBC9E1FFECC9E2FF040EE66EE9C91C
:101E940000F0EAC901F041EC05F0010E006E3CD0FF
:101EA400010E0B01AA5F000EAB5BAC5BAD5BDBD735
:101EB40007C1AAFB08C1ABFB09C1ACFB0AC1ADFB5E
:101EC4009EB623D001010751081109110A111CE023
:101ED4000B01AA51AB11AC11AD110FE1EBC9E1FF3C
:101EE400ECC9E2FF040EE66EE9C900F0EAC901F0AC
:101EF40041EC05F0010E006E0FD0010E0B01AA5F3C
:101F0400000EAB5BAC5BAD5BDBD7C5BC02D0006A3B
:0A1F140003D0C584020E006E120017
:101F1E0007C1ABFB08C1ACFB09C1ADFB0AC1AEFBEF
:101F2E000B01A96BAA6BAA51120802E1A9518E08E6
:101F3E0009E334EC05F0005201E004D00B01A94B8B
:101F4E00AA2BF1D70B01120EAA5D02E18F0EA95D2D
:101F5E0003E37B0E006E27D0C580C5A023D0010100
:101F6E000751081109110A111CE00B01AB51AC11FC
:101F7E00AD11AE110FE1EBC9E1FFECC9E2FF050EA9
:101F8E00E66EE9C900F0EAC901F041EC05F0010E78
:101F9E00006E09D0010E0B01AB5F000EAC5BAD5BAA
:081FAE00AE5BDBD7006A1200F4
:101FB600086A096A100E0C6E013408360936045098
:101FC600085E0550D8A0053C095ED8B007D004507D
:101FD60008260550D8B0053C0926D89000360136AB
:061FE6000C2EEAD71200E8
:101FEC00020E0C6E080E0D6E0D2EFED70C2EFCD7AD
:041FFC0000001200CF
:0A200000050E0D6E0D2EFED7120026
:10200A0083CBF6FF84CBF7FF85CBF8FF0900F5CF2A
:10201A0000F0005218E083CBF6FF84CBF7FF85CBA4
:10202A00F8FF0900F5CF00F081CBE1FF82CBE2FF98
:10203A0000C0E6FF0B01814B822B010E8327000EA5
:10204A0084238523DDD781CBE1FF82CBE2FFE66AD9
:02205A00120072
:10205C000B01826B815109081DE20A0E046E81CBC3
:10206C0000F025EC05F000C082FB00C082FB82373B
:10207C0082918237829182378291823782910A0EC5
:10208C00046E81CB00F025EC05F008C000F0005088
:0E209C00821302D081CB82FB82CB00F01200B7
:1020AA0039DFD00E0B01A96FD0DE81CBA9FBCDDEC3
:1020BA0047EC09F0D10E0B01A96FC7DE0B01A96B22
:1020CA0026EC0AF000C082FBBEDE82CB00F01200D2
:1020DA0081CB04F082CB05F00B018551861124E0F7
:1020EA00010E855F000E865B04C002F005C003F096
:1020FA00044A052A83CB00F084CB01F0834B842B5E
:10210A0000C0E9FF01C0EAFF02C0E1FF03C0E2FF2D
:10211A00EECFE6FF02C0E9FF03C0EAFFEECF00F010
:10212A00005201E101D0D8D785CB00F086CB01F06F
:10213A00010E855F000E865B0050011008E004C0A6
:10214A00E1FF05C0E2FFE66A044A052AEDD781CB22
:08215A0000F082CB01F012003D
:102162000D0E0B01B76FBDEC01F00A0E0B01B76F3C
:06217200BDEC01F01200BB
:102178000B01816B826B800E8219006E800E005CF1
:1021880002E1080E815D1AE28151010FA96FAA6B65
:10219800AB6BAC6BAD6BAE6BAF6BB06BB16BB26B6B
:1021A800B36BB46BB56BFCEC05F06A0E0D6E0D2EBF
:0E21B800FED700000B01814B822BDDD71200F9
:1021C60081CBF6FF82CBF7FF83CBF8FF0900F5CF73
:1021D60000F0005212E081CBF6FF82CBF7FF83CBF3
:1021E600F8FF0900F5CFB7FBBDEC01F0010E0B01BE
:1021F6008127000E82238323E3D71A0E0D6E0D2E40
:06220600FED700001200EB
:10220C0081CB00F00032009E0032009E0032009E16
:10221C000032009E0A0E0002F3CF01F00F0E0B01EC
:0A222C008115006E0150002612001B
:10223600A69C82CBAAFF81CBA9FFA69EA680A8CF8B
:0422460000F0120092
:10224A00020E0C6E9D0E0D6E0D2EFED70C2EFCD7B7
:06225A000000000012006C
:102260000B01846B81CBE9FF82CBEAFFEECF83FBCE
:102270008351000A0FE083CBB7FBBDEC01F00B01EB
:10228000842B84518125E96E000E8221EA6EEECF07
:0622900083FBEED71200F3
:10229600800E0B01826F836B846B300E856F300E60
:1022A600866F300E876F300E886F300E896F300E56
:1022B6008A6F300E8B6F300E8C6F8D6B800E84198B
:1022C600006E800E005C02E1080E835D3AE20001BA
:1022D6007D51000A19E10B0182518115016E0150F1
:1022E600000809E2850E8325E16E0B0E8421E26E5D
:1022F600310EE66E08D0850E8325E16E0B0E842125
:10230600E26E300EE66E18D00B0182518115016E19
:102316000150000809E2850E8325E16E0B0E84212B
:10232600E26E2A0EE66E08D0850E8325E16E0B0E50
:102336008421E26E2E0EE66E8233829F834B842BBF
:0E234600BDD78D6B850E006E0B0E016E120062
:10235400E4DDD00E0B01A96F7BDD81CBA9FB78DD19
:0A23640082CBA9FB75DD72DD1200CB
:10236E0081CBE9FF82CBEAFFEECF83FB000E0B01A0
:10237E00846F000E846F000E841902E1200E831903
:10238E0007E0000E841902E1090E831901E003D063
:10239E00814B822BE5D7856B866B876B886B000E26
:1023AE00841902E12D0E831905E1874B882B814B91
:1023BE00822B08D0000E841902E12B0E831902E144
:1023CE00814B822B81CBE9FF82CBEAFFEECF83FBE1
:1023DE00000E846F000E846F83CBA9FBF2EC09F024
:1023EE00005219E085CB00F086CB01F00A0E046E88
:1023FE00000E056EFEEC09F0300E835D026E000ECF
:10240E008459036E02500024856F03500120866F9D
:10241E00814B822BD7D78751881108E08551000850
:10242E00006E86CB01F0000E015604D085CB00F075
:06243E0086CB01F0120044
:102444000B0E0C6E570E0D6E0D2EFED70C2EFCD7F8
:0624540000000000120070
:10245A000B01A16BA26B956B966B83CB00F084CBBF
:10246A0001F085CB02F0010E8327000E8423852319
:10247A0000C0F6FF01C0F7FF02C0F8FF0900F5CF60
:10248A0000F000C092FB0052D8B43BEF22F0925108
:10249A00250A0BE081CBE1FF82CBE2FF92CBE6FF7C
:1024AA00814B822BA14BA22BD8D7936B946B956B44
:1024BA00966B23D09587010E8327000E84238523EC
:1024CA0059D09581010E8327000E8423852352D08B
:1024DA009583010E8327000E842385234BD096878C
:1024EA00010E8327000E8423852344D09585010E8F
:1024FA008327000E842385233DD083CBF6FF84CB2C
:10250A00F7FF85CBF8FF0900F5CF01F001502D0A3E
:10251A00D1E083CBF6FF84CBF7FF85CBF8FF090028
:10252A00F5CF01F00150200ACCE083CBF6FF84CB33
:10253A00F7FF85CBF8FF0900F5CF01F001502B0A10
:10254A00C7E083CBF6FF84CBF7FF85CBF8FF090002
:10255A00F5CF01F00150230AC2E083CBF6FF84CB0A
:10256A00F7FF85CBF8FF0900F5CF01F00150300ADB
:10257A00BDE001D09ED795A301D0959195A701D032
:10258A00959583CBF6FF84CBF7FF85CBF8FF09003F
:10259A00F5CF00F0000E016E00C0A9FBF2EC09F0C5
:1025AA00005236E0936B946B93CB00F094CB01F01E
:1025BA000A0E046E000E056EFEEC09F083CBF6FFE0
:1025CA0084CBF7FF85CBF8FF0900F5CF02F0025064
:1025DA000024936F000E0120946F300E935F000E5B
:1025EA00945B010E8327000E8423852383CBF6FF99
:1025FA0084CBF7FF85CBF8FF0900F5CF00F0000E7A
:10260A00016E00C0A9FBF2EC09F00052CDE133D013
:10261A0083CBF6FF84CBF7FF85CBF8FF0900F5CF14
:10262A0001F001502A0A27E186CBE9FF87CBEAFFAE
:10263A00EECF00F0EECF01F000C0E9FF01C0EAFFE3
:10264A00EECF93FBEECF94FB86CBE9FF87CBEAFF75
:10265A00020EEE24006E000EEE20016E86CBE1FF24
:10266A0087CBE2FF00C0E6FF01C0E6FF010E832729
:10267A00000E8423852383CBF6FF84CBF7FF85CB1B
:10268A00F8FF0900F5CF01F001502E0A70E1010EA2
:10269A008327000E8423852383CBF6FF84CBF7FFA1
:1026AA0085CBF8FF0900F5CF01F001502A0A28E18D
:1026BA0086CBE9FF87CBEAFFEECF00F0EECF01F041
:1026CA0000C0E9FF01C0EAFFEECF90FBEECF91FB1D
:1026DA0086CBE9FF87CBEAFF020EEE24006E000EDE
:1026EA00EE20016E86CBE1FF87CBE2FF00C0E6FF5A
:1026FA0001C0E6FF010E8327000E8423852336D00E
:10270A00906B916B83CBF6FF84CBF7FF85CBF8FFF9
:10271A000900F5CF00F0000E016E00C0A9FBF2EC33
:10272A0009F0005223E090CB00F091CB01F00A0EA1
:10273A00046E000E056EFEEC09F083CBF6FF84CB27
:10274A00F7FF85CBF8FF0900F5CF02F0025000240D
:10275A00906F000E0120916F300E905F000E915B1A
:10276A00010E8327000E84238523CCD703D0906BD8
:10277A00916B968983CB00F084CB01F085CB02F074
:10278A00010E8327000E8423852300C0F6FF01C0B3
:10279A00F7FF02C0F8FF0900F5CF92FBF9D0A1CBF1
:1027AA0000F0A2CB01F03FEF22F09589E3D796859E
:1027BA002ED1958B96812BD1968329D1958D27D1B0
:1027CA0026D1958B958F23D186CBE9FF87CBEAFF5C
:1027DA00EECF00F0EECF01F000C0E9FF01C0EAFF42
:1027EA00EECF9DFBEECF9EFB86CBE9FF87CBEAFFC0
:1027FA00020EEE24006E000EEE20016E86CBE1FF83
:10280A0087CBE2FF00C0E6FF01C0E6FF000E9E197B
:10281A0002E1000E9D1904E1110E9D6F090E9E6FD3
:10282A009F6BA06B9F519D25E96EA0519E21EA6E78
:10283A00EE520BE0010E9F25006E000EA021016EE4
:10284A0000C09FFB01C0A0FBEDD7905191110AE097
:10285A00A051915D02E19F51905D04E290CB9FFBF4
:10286A0091CBA0FB9451A05D02E193519F5D05E2DB
:10287A009F51935FA051945B02D0936B946B95B771
:10288A0016D093CB00F094CB01F0010E935F000EAB
:10289A00945B005001100BE081CBE1FF82CBE2FF99
:1028AA00200EE66E814B822BA14BA22BEAD79FCB3F
:1028BA0002F0A0CB03F0010E9F5D006E000EA0593E
:1028CA00016E00C09FFB01C0A0FB0250031019E07B
:1028DA009DCBE9FF9ECBEAFF81CBE1FF82CBE2FFF2
:1028EA00EECFE6FF814B822B010E9D25006E000E76
:1028FA009E21016E00C09DFB01C09EFBA14BA22B35
:10290A00D6D795A716D093CB00F094CB01F0010E41
:10291A00935F000E945B005001100BE081CBE1FF46
:10292A0082CBE2FF200EE66E814B822BA14BA22BBB
:10293A00EAD793D586CBE9FF87CBEAFFEECF00F043
:10294A00EECF01F000C0E9FF01C0EAFFEECF92FB33
:10295A0086CBE9FF87CBEAFF020EEE24006E000E5B
:10296A00EE20016E86CBE1FF87CBE2FF00C0E6FFD7
:10297A0001C0E6FF920E9D6F0B0E9E6F010E9F6FB8
:10298A00000EA06F62D7C00E9513000E96133FD0AB
:10299A009251000AD8B403D792516C0AD8B405D719
:1029AA0092514C0AD8B401D79251660AD8B4FFD6CC
:1029BA009251450AD8B4FDD69251650AD8B4FAD6CE
:1029CA009251670AD8B4F8D692516F0AD8B4F6D69B
:1029DA009251640AD8B4F4D69251690AD8B4F0D69E
:1029EA009251700AD8B4EDD69251580AD8B4E9D6A1
:1029FA009251780AD8B4E6D69251730AD8B4E4D67A
:102A0A009251630A97E09251750ABDE0B3D7000E5E
:102A1A009515006E9651070B016E00500110D8B43F
:102A2A00E2EF1DF096A904D0060E906F000E916F8A
:102A3A0086CBE9FF87CBEAFFEECF00F0EECF01F0BD
:102A4A0000C0E9FF01C0EAFFEECF97FBEECF98FB8B
:102A5A00EECF99FBEECF9AFB86CBE9FF87CBEAFF55
:102A6A00040EEE24006E000EEE20016E86CBE1FF0E
:102A7A0087CBE2FF00C0E6FF01C0E6FF046A056AF1
:102A8A00066A076A97CB00F098CB01F099CB02F05F
:102A9A009ACB03F074EC09F0010ED8B0000E006E68
:102AAA00005205E0997F030E9513000E96139B6B57
:102ABA009C6B97CB00F098CB01F099CB02F09ACBA4
:102ACA0003F0046A056A066A076ADBEC09F0000E7D
:102ADA00D8A4010E006E0052D8B48AD09ACB00F066
:102AEA00016A026A036AFF0E0016000E01167E0EC4
:102AFA00005E000E015A00C09BFB01C09CFB010E48
:102B0A00005E000E015A00C09BFB01C09CFB030E35
:102B1A00046E000E056EFEEC09F000C09BFB01C0BE
:102B2A009CFB0A0E046E000E056E8CEC0AF000C0C7
:102B3A009BFB01C09CFB800E0118026E800E025C9A
:102B4A0002E1000E005C05E2010E0B019B5F000E24
:102B5A009C5B0B019B510008A96FF0EC0AF097CB24
:102B6A0004F098CB05F099CB06F09ACB07F006EC67
:102B7A0004F000C09DFB01C09EFB02C09FFB03C086
:102B8A00A0FB000E046E000E056E000E066E7F0E90
:102B9A00076E9DCB00F09ECB01F09FCB02F0A0CB3D
:102BAA0003F074EC09F0010ED8B0000E006E00526A
:102BBA0005E0010E9B5F000E9C5B1AD0000E046EAE
:102BCA00000E056E200E066E820E076E9DCB00F07B
:102BDA009ECB01F09FCB02F0A0CB03F074EC09F07E
:102BEA00000ED8B0010E006E005202E09B4B9C2BE7
:102BFA00800E006E800E9C19005C02E19B51000859
:102C0A0003E3010E926F02D09BCB92FB96B118D0D0
:102C1A0096A315D0800E9C19006E7F0E005C02E10F
:102C2A00FC0E9B5D0BE3800E9C19006E800E9119C1
:102C3A00005C02E190519B5D01E201D001D0EFD32B
:102C4A009051911106E096A304D0010E905F000EF8
:102C5A00915B9151000802E19051080803E2080EC5
:102C6A00926F02D090CB92FB97CB00F098CB01F0F9
:102C7A0099CB02F09ACB03F0046A056A066A076ADE
:102C8A00DBEC09F0000ED8A4010E006E0052D8B495
:102C9A004BD19BCBA9FBF0EC0AF000C004F001C0B9
:102CAA0005F002C006F003C007F097CB00F098CBFE
:102CBA0001F099CB02F09ACB03F0CEEC0DF000C0F4
:102CCA0097FB01C098FB02C099FB03C09AFB0B015A
:102CDA0092510008A96FF0EC0AF000C004F001C09C
:102CEA0005F002C006F003C007F097CB00F098CBBE
:102CFA0001F099CB02F09ACB03F0CEEC0DF000C0B4
:102D0A00A3FB01C0A4FB02C0A5FB03C0A6FBA3CB87
:102D1A0097FBA4CB98FBA5CB99FBA6CB9AFBA3CB9D
:102D2A0000F0A4CB01F0A5CB02F0A6CB03F08CEC0B
:102D3A000EF04DEC05F000C004F001C005F002C031
:102D4A0006F003C007F0A3CB00F0A4CB01F0A5CB9B
:102D5A0002F0A6CB03F0F8EC05F0000E046E000EAC
:102D6A00056E000E066E7E0E076E74EC09F0000EFC
:102D7A00D8B0010E006E00521AE097CB00F098CB43
:102D8A0001F099CB02F09ACB03F0000E046E000E0C
:102D9A00056E000E066E7E0E076EF6EC01F000C0A0
:102DAA0097FB01C098FB02C099FB03C09AFB97CB23
:102DBA0000F098CB01F099CB02F09ACB03F08CEC9F
:102DCA000EF00B019251010F096E0A6A000E0A22D7
:102DDA0009C004F00AC005F0000E0ABEFF0E066E16
:102DEA00076E043604900536063607360436049014
:102DFA00053606360736590E0424F66E810E05206E
:102E0A00F76E000E0620F86E0900F5CF05F00900EE
:102E1A00F5CF06F00900F5CF07F00900F5CF08F065
:102E2A000850035C08E10750025C05E10650015CAA
:102E3A0002E10550005C1EE30B0197CB00F098CB32
:102E4A0001F099CB02F09ACB03F0CD0E046ECC0EB2
:102E5A00056E4C0E066E7B0E076E06EC04F000C083
:102E6A0097FB01C098FB02C099FB03C09AFB9B4BDE
:102E7A009C2B5AD097CB00F098CB01F099CB02F05B
:102E8A009ACB03F08CEC0EF092CB04F0000E056E98
:102E9A00066E076E04360490053606360736043683
:102EAA000490053606360736590E0424F66E810E4E
:102EBA000520F76E000E0620F86E0900F5CF05F022
:102ECA000900F5CF06F00900F5CF07F00900F5CFA4
:102EDA0008F00850035C08E10750025C05E106505F
:102EEA00015C02E10550005C1FE20B0197CB00F088
:102EFA0098CB01F099CB02F09ACB03F0000E046E46
:102F0A00000E056E200E066E820E076E06EC04F0A9
:102F1A0000C097FB01C098FB02C099FB03C09AFB53
:102F2A00010E9B5F000E9C5B0B0196A393D096B794
:102F3A0091D0800E000A006E800E9119005C02E1A9
:102F4A0090510A0804E20A0E906F000E916F97CB17
:102F5A0000F098CB01F099CB02F09ACB03F08CECFD
:102F6A000EF000C09DFB01C09EFB02C09FFB03C088
:102F7A00A0FB9D519E119F11A01142E00A0E046E02
:102F8A00000E056E066E076E9DCB00F09ECB01F01B
:102F9A009FCB02F0A0CB03F056EC06F008C000F07D
:102FAA0009C001F00AC002F00BC003F0000E046E63
:102FBA00031808E10450021805E10450011802E15F
:102FCA000050000A1DE1010E905F000E915B0A0E8F
:102FDA00046E000E056E066E076E9DCB00F09ECB4A
:102FEA0001F09FCB02F0A0CB03F056EC06F000C034
:102FFA009DFB01C09EFB02C09FFB03C0A0FBB9D78B
:10300A00800E9119006E800E005C02E19251905D73
:10301A0021E29051925DA96FF0EC0AF000C004F031
:10302A0001C005F002C006F003C007F097CB00F01C
:10303A0098CB01F099CB02F09ACB03F0CEEC0DF0CD
:10304A0000C097FB01C098FB02C099FB03C09AFB22
:10305A0090CB92FB050E0B019025006E000E91217C
:10306A00016E0050935F0150945B9051911103E1FE
:10307A0096B701D004D0010E935F000E945B030E45
:10308A009515006E96CB01F0000E01160050011046
:10309A0004E0010E935F000E945B95A539D095A3C9
:1030AA0012D095A103D02D0E886F02D02B0E886FF7
:1030BA0081CBE1FF82CBE2FF88CBE6FF814B822BFB
:1030CA00A14BA22B0CD095A10AD081CBE1FF82CBD8
:1030DA00E2FF200EE66E814B822BA14BA22B800EC3
:1030EA00006E800E9419005C02E1935100080FE211
:1030FA0081CBE1FF82CBE2FF300EE66E814B822B61
:10310A00A14BA22B010E935F000E945BE8D73AD035
:10311A0095B718D0800E006E800E9419005C02E1FB
:10312A00935100080FE281CBE1FF82CBE2FF200E30
:10313A00E66E814B822BA14BA22B010E935F000EF0
:10314A00945BE8D795A312D095A103D02D0E896F71
:10315A0002D02B0E896F81CBE1FF82CBE2FF89CBB4
:10316A00E6FF814B822BA14BA22B0CD095A10AD052
:10317A0081CBE1FF82CBE2FF200EE66E814B822BF0
:10318A00A14BA22B97CB00F098CB01F099CB02F080
:10319A009ACB03F08CEC0EF000C09DFB01C09EFBA5
:1031AA0002C09FFB03C0A0FB92CB00F0000E016E91
:1031BA00026E036E00360090013602360336003680
:1031CA000090013602360336590E0024F66E810E3F
:1031DA000120F76E000E0220F86E0900F5CF04F008
:1031EA000900F5CF05F00900F5CF06F00900F5CF83
:1031FA0007F09DCB00F09ECB01F09FCB02F0A0CB55
:10320A0003F056EC06F0300E002681CBE1FF82CBAC
:10321A00E2FF00C0E6FF814B822BA14BA22B90510B
:10322A00911103E196B701D06FD081CBE1FF82CB38
:10323A00E2FF2E0EE66E814B822BA14BA22B9251FE
:10324A00905F000E915B92534DE0920792CB00F093
:10325A00000E016E026E036E0036009001360236D1
:10326A00033600360090013602360336590E002422
:10327A00F66E810E0120F76E000E0220F86E09002C
:10328A00F5CF04F00900F5CF05F00900F5CF06F0F7
:10329A000900F5CF07F09DCB00F09ECB01F09FCB44
:1032AA0002F0A0CB03F056EC06F00A0E046E000EF4
:1032BA00056E066E076E56EC06F008C000F009C0EF
:1032CA0001F00AC002F00BC003F0300E002681CBD9
:1032DA00E1FF82CBE2FF00C0E6FF814B822BA14BCC
:1032EA00A22BB1D7905191110FE081CBE1FF82CB94
:1032FA00E2FF300EE66E814B822BA14BA22B010E10
:10330A00905F000E915BEED795AB0BD081CBE1FFBE
:10331A0082CBE2FF450EE66E814B822BA14BA22B9C
:10332A000AD081CBE1FF82CBE2FF650EE66E814BCC
:10333A00822BA14BA22B800E9C19006E800E005C82
:10334A0002E1000E9B5D11E29B5100089B6F9C51AC
:10335A00000E9C5781CBE1FF82CBE2FF2D0EE66E79
:10336A00814B822BA14BA22B0AD081CBE1FF82CBCE
:10337A00E2FF2B0EE66E814B822BA14BA22B0A0E8B
:10338A00046E000E056E9BCB00F09CCB01F08CEC1A
:10339A000AF0300E002681CBE1FF82CBE2FF00C0AB
:1033AA00E6FF0B01814B822BA14BA22B0A0E046E66
:1033BA00000E056E9BCB00F09CCB01F08CEC0AF062
:1033CA0008C000F009C001F0300E002681CBE1FFF1
:1033DA0082CBE2FF00C0E6FF0B01814B822BA14B9F
:1033EA00A22B95A71AD0800E006E800E9419005C4D
:1033FA0002E19351000811E281CBE1FF82CBE2FFA7
:10340A00200EE66E814B822BA14BA22B010E935FFD
:10341A00000E945B93519411EFE132EF12F096A3F0
:10342A00F3D0800E9C19006E800E005C02E1000E43
:10343A009B5D0AE2010E9B5D006E000E9C59016EB7
:10344A000050905F0150915B97CB00F098CB01F050
:10345A0099CB02F09ACB03F08CEC0EF000C09DFBE6
:10346A0001C09EFB02C09FFB03C0A0FB010E926F2E
:10347A0092510A0A34E092CB00F0000E016E026EFD
:10348A00036E00360090013602360336003600908D
:10349A00013602360336590E0024F66E810E0120DB
:1034AA00F76E000E0220F86E0900F5CF01F0090050
:1034BA00F5CF02F00900F5CF03F00900F5CF04F0CB
:1034CA000450A05D08E103509F5D05E102509E5D36
:1034DA0002E101509D5D01E202D0922BC9D79251BF
:1034EA00905DA76F000E9159A86FA7CB90FBA8CB50
:1034FA0091FB9DCB00F09ECB01F09FCB02F0A0CBBD
:10350A0003F04DEC05F000C004F001C005F002C064
:10351A0006F003C007F097CB00F098CB01F099CBE7
:10352A0002F09ACB03F0F8EC05F000C0A3FB01C04F
:10353A00A4FB02C0A5FB03C0A6FBA7CBA9FBF0EC2A
:10354A000AF0A3CB04F0A4CB05F0A5CB06F0A6CBDA
:10355A0007F006EC04F0000E046E000E056E000E75
:10356A00066E7E0E076EF6EC01F08CEC0EF000C0D3
:10357A009DFB01C09EFB02C09FFB03C0A0FB9051B4
:10358A00911142E00A0E046E000E056E066E076E79
:10359A009DCB00F09ECB01F09FCB02F0A0CB03F0B5
:1035AA0056EC06F008C000F009C001F00AC002F0AB
:1035BA000BC003F0000E046E031808E10450021851
:1035CA0005E10450011802E10050000A1DE10A0E4B
:1035DA00046E000E056E066E076E9DCB00F09ECB44
:1035EA0001F09FCB02F0A0CB03F056EC06F000C02E
:1035FA009DFB01C09EFB02C09FFB03C0A0FB010E06
:10360A00905F000E915BBBD7800E006E800E911901
:10361A00005C02E190510C0816E390CBA9FBCCECBC
:10362A0007F097CB04F098CB05F099CB06F09ACB2C
:10363A0007F0F6EC01F000C097FB01C098FB02C04E
:10364A0099FB03C09AFB97CB00F098CB01F099CB7A
:10365A0002F09ACB03F0046A056A066A076ADBEC91
:10366A0009F0000ED8A4010E006E0052D8B477D02B
:10367A0097CB00F098CB01F099CB02F09ACB03F0EC
:10368A008CEC0EF0000E046E031808E104500218C8
:10369A0005E10450011802E10050000A60E1800EC1
:1036AA00006E800E9C19005C02E19B51010857E2F2
:1036BA009BCBA9FBF0EC0AF000C004F001C005F0B6
:1036CA0002C006F003C007F097CB00F098CB01F0D8
:1036DA0099CB02F09ACB03F0CEEC0DF05F0E046E9C
:1036EA00700E056E090E066E810E076E74EC09F0F7
:1036FA00010ED8B0000E006E005206E0090E0B0152
:10370A009B5F000E9C5B05D00B01080E9B5F000EB1
:10371A009C5B9BCBA9FBF0EC0AF000C004F001C053
:10372A0005F002C006F003C007F097CB00F098CB73
:10373A0001F099CB02F09ACB03F0CEEC0DF08CECB1
:10374A000EF000C09DFB01C09EFB02C09FFB03C0A0
:10375A00A0FB0B01976B986B996B9A6B38D097CB40
:10376A0000F098CB01F099CB02F09ACB03F08CECE5
:10377A000EF000C09DFB01C09EFB02C09FFB03C070
:10378A00A0FB9DCB00F09ECB01F09FCB02F0A0CB1B
:10379A0003F04DEC05F000C004F001C005F002C0D2
:1037AA0006F003C007F097CB00F098CB01F099CB55
:1037BA0002F09ACB03F0F8EC05F000C097FB01C0C9
:1037CA0098FB02C099FB03C09AFB9B6B9C6B010E92
:1037DA00926F92510A0A34E092CB00F0000E016E09
:1037EA00026E036E0036009001360236033600364A
:1037FA000090013602360336590E0024F66E810E09
:10380A000120F76E000E0220F86E0900F5CF01F0D4
:10381A000900F5CF02F00900F5CF03F00900F5CF52
:10382A0004F00450A05D08E103509F5D05E10250D9
:10383A009E5D02E101509D5D01E202D0922BC9D743
:10384A0092519025006E000E9121016E9B51002627
:10385A009C5101220050935F0150945B96B704D0AB
:10386A009051911101E104D0010E935F000E945B17
:10387A00030E9515006E96CB01F0000E011600504E
:10388A00011004E0010E935F000E945B95A539D0F8
:10389A0095A312D095A103D02D0E8A6F02D02B0EBC
:1038AA008A6F81CBE1FF82CBE2FF8ACBE6FF814BB5
:1038BA00822BA14BA22B0CD095A10AD081CBE1FF80
:1038CA0082CBE2FF200EE66E814B822BA14BA22B0C
:1038DA00800E006E800E9419005C02E1935100087C
:1038EA000FE281CBE1FF82CBE2FF300EE66E814B25
:1038FA00822BA14BA22B010E935F000E945BE8D79B
:10390A003AD095B718D0800E006E800E9419005CDC
:10391A0002E1935100080FE281CBE1FF82CBE2FF83
:10392A00200EE66E814B822BA14BA22B010E935FD8
:10393A00000E945BE8D795A312D095A103D02D0E63
:10394A008B6F02D02B0E8B6F81CBE1FF82CBE2FF14
:10395A008BCBE6FF814B822BA14BA22B0CD095A1DE
:10396A000AD081CBE1FF82CBE2FF200EE66E814BCB
:10397A00822BA14BA22B92CB00F0920700524CE073
:10398A0092CB00F0000E016E026E036E00360090BC
:10399A000136023603360036009001360236033607
:1039AA00590E0024F66E810E0120F76E000E0220D9
:1039BA00F86E0900F5CF04F00900F5CF05F009000B
:1039CA00F5CF06F00900F5CF07F09DCB00F09ECBAE
:1039DA0001F09FCB02F0A0CB03F056EC06F00A0EE2
:1039EA00046E000E056E066E076E56EC06F008C0F1
:1039FA0000F009C001F00AC002F00BC003F0300E5B
:103A0A00002681CBE1FF82CBE2FF00C0E6FF814BBB
:103A1A00822BA14BA22BAFD7800E006E800E9C1971
:103A2A00005C02E19B5100080FE281CBE1FF82CBEF
:103A3A00E2FF300EE66E814B822BA14BA22B010EC8
:103A4A009B5F000E9C5BE8D7800E000A006E800E1A
:103A5A009119005C02E19051080803E2080E926F86
:103A6A0002D090CB92FB9251905F000E915B9253E1
:103A7A0003E196B701D00AD081CBE1FF82CBE2FF06
:103A8A002E0EE66E814B822BA14BA22B92CBA9FB69
:103A9A00F0EC0AF097CB04F098CB05F099CB06F03E
:103AAA009ACB07F006EC04F060EC05F000C09DFB31
:103ABA0001C09EFB02C09FFB03C0A0FB92534DE0D6
:103ACA00920792CB00F0000E016E026E036E003672
:103ADA00009001360236033600360090013602366F
:103AEA000336590E0024F66E810E0120F76E000E81
:103AFA000220F86E0900F5CF04F00900F5CF05F0B1
:103B0A000900F5CF06F00900F5CF07F09DCB00F0CC
:103B1A009ECB01F09FCB02F0A0CB03F056EC06F04F
:103B2A000A0E046E000E056E066E076E56EC06F05F
:103B3A0008C000F009C001F00AC002F00BC003F08F
:103B4A00300E002681CBE1FF82CBE2FF00C0E6FF08
:103B5A00814B822BA14BA22BB1D7905191110FE02F
:103B6A0081CBE1FF82CBE2FF300EE66E814B822BE6
:103B7A00A14BA22B010E905F000E915BEED795A789
:103B8A001AD0800E006E800E9419005C02E19351E7
:103B9A00000811E281CBE1FF82CBE2FF200EE66E44
:103BAA00814B822BA14BA22B010E935F000E945BDB
:103BBA0093519411EFE132EF12F0C00E9515016E98
:103BCA0096CB02F0000E0216000E021802E1000E59
:103BDA000118D8A480D095A927D086CBE9FF87CB36
:103BEA00EAFFEECF00F0EECF01F000C0E9FF01C01E
:103BFA00EAFFEECF9DFBEECF9EFBEECF9FFBEECF13
:103C0A00A0FB86CBE9FF87CBEAFF040EEE24006E09
:103C1A00000EEE20016E86CBE1FF87CBE2FF00C0EB
:103C2A00E6FF01C0E6FF2FD086CBE9FF87CBEAFF8C
:103C3A00EECF00F0EECF01F000C0E9FF01C0EAFFCD
:103C4A00EECF00F0EECF01F0000E01BEFF0E026EC5
:103C5A00036E00C09DFB01C09EFB02C09FFB03C018
:103C6A00A0FB86CBE9FF87CBEAFF020EEE24006EAB
:103C7A00000EEE20016E86CBE1FF87CBE2FF00C08B
:103C8A00E6FF01C0E6FF800EA019006E800E005C00
:103C9A0008E1000E9F5D05E1000E9E5D02E1000E47
:103CAA009D5D18E2030E9513000E9613006A016AD1
:103CBA00026A036A9D51005E9E51015A9F51025A3F
:103CCA00A051035A00C09DFB01C09EFB02C09FFB8E
:103CDA0003C0A0FB4ED095A927D086CBE9FF87CB9E
:103CEA00EAFFEECF00F0EECF01F000C0E9FF01C01D
:103CFA00EAFFEECF9DFBEECF9EFBEECF9FFBEECF12
:103D0A00A0FB86CBE9FF87CBEAFF040EEE24006E08
:103D1A00000EEE20016E86CBE1FF87CBE2FF00C0EA
:103D2A00E6FF01C0E6FF25D086CBE9FF87CBEAFF95
:103D3A00EECF00F0EECF01F000C0E9FF01C0EAFFCC
:103D4A00EECF9DFBEECF9EFB000E9F6FA06F86CB42
:103D5A00E9FF87CBEAFF020EEE24006E000EEE208A
:103D6A00016E86CBE1FF87CBE2FF00C0E6FF01C010
:103D7A00E6FF000E911902E1000E90190FE1000E04
:103D8A00006EA01908E100509F1905E100509E1924
:103D9A0002E19D51000A02E1904B912BC00E95154C
:103DAA00006E00C005F0AED0010E926F92510A0A61
:103DBA0034E092CB00F0000E016E026E036E003604
:103DCA00009001360236033600360090013602367C
:103DDA000336590E0024F66E810E0120F76E000E8E
:103DEA000220F86E0900F5CF01F00900F5CF02F0C4
:103DFA000900F5CF03F00900F5CF04F00450A05DE7
:103E0A0008E103509F5D05E102509E5D02E1015009
:103E1A009D5D01E202D0922BC9D782D0010E926F2A
:103E2A009251080A34E092CB00F0000E016E026E45
:103E3A00036E0036009001360236033600360090D3
:103E4A00013602360336170E0024F66E820E012062
:103E5A00F76E000E0220F86E0900F5CF01F0090096
:103E6A00F5CF02F00900F5CF03F00900F5CF04F011
:103E7A000450A05D08E103509F5D05E102509E5D7C
:103E8A0002E101509D5D01E202D0922BC9D748D0D0
:103E9A00010E926F92510C0A34E092CB00F0000EA0
:103EAA00016E026E036E003600900136023603364A
:103EBA00003600900136023603361B0E0024F66ED9
:103ECA00800E0120F76E000E0220F86E0900F5CF71
:103EDA0001F00900F5CF02F00900F5CF03F009005F
:103EEA00F5CF04F00450A05D08E103509F5D05E1A1
:103EFA0002509E5D02E101509D5D01E202D0922BCB
:103F0A00C9D70ED00550000AD8B44ED70550C00AFA
:103F1A00D8B44AD70550800A81E00550400AB8E073
:103F2A00800E006E800E9119005C02E19051925D44
:103F3A0003E290CB92FB0DD0800E9119006E800E99
:103F4A00005C02E19251905D04E292CB90FB000E7C
:103F5A00916F935194110EE0030E9515006E96CB56
:103F6A0001F0000E01160050011004E0010E935FEB
:103F7A00000E945B800E9119006E800E9419005CFD
:103F8A0002E19351905D05E29051935F9151945BE8
:103F9A0002D0936B946BC40E9515016E9651080B63
:103FAA00026E0250080A02E1400E011808E193511C
:103FBA00941104E0010E935F000E945B1CD0C00EB6
:103FCA009515016E9651080B026E0250080A02E11D
:103FDA00800E011810E1800E006E800E9419005CAC
:103FEA0002E19351020805E2020E935F000E945B10
:103FFA0002D0936B946B95A55DD095A312D095A131
:10400A0003D02D0E8C6F02D02B0E8C6F81CBE1FF6B
:10401A0082CBE2FF8CCBE6FF814B822BA14BA22BFA
:10402A0034D095A10BD081CBE1FF82CBE2FF200EE9
:10403A00E66E814B822BA14BA22B27D0C00E951581
:10404A00016E9651080B026E0250080A02E1800EB8
:10405A0001181BE181CBE1FF82CBE2FF300EE66E55
:10406A00814B822BA14BA22B95AB03D0580E8D6F9F
:10407A0002D0780E8D6F81CBE1FF82CBE2FF8DCB30
:10408A00E6FF814B822BA14BA22B9351941111E095
:10409A0081CBE1FF82CBE2FF300EE66E814B822BB1
:1040AA00A14BA22B010E935F000E945B93519411C6
:1040BA00EFE174D09351941113E095B711D081CBED
:1040CA00E1FF82CBE2FF200EE66E814B822BA14BF1
:1040DA00A22B010E935F000E945B93519411EFE1B2
:1040EA0095A312D095A103D02D0E8E6F02D02B0E60
:1040FA008E6F81CBE1FF82CBE2FF8ECBE6FF814B55
:10410A00822BA14BA22B0CD095A10AD081CBE1FF27
:10411A0082CBE2FF200EE66E814B822BA14BA22BB3
:10412A00C00E9515016E9651080B026E0250080AD0
:10413A0002E1400E01180BE181CBE1FF82CBE2FFE5
:10414A00300EE66E814B822BA14BA22B27D0C00EDC
:10415A009515016E9651080B026E0250080A02E18B
:10416A00800E01181BE181CBE1FF82CBE2FF300E0A
:10417A00E66E814B822BA14BA22B95AB03D0580E36
:10418A008F6F02D0780E8F6F81CBE1FF82CBE2FF77
:10419A008FCBE6FF814B822BA14BA22B800E006EA8
:1041AA00800E9119005C02E19051925D0BE281CB85
:1041BA00E1FF82CBE2FF300EE66E814B822BA14BF0
:1041CA00A22BECD790CB00F091CB01F0010E905FBF
:1041DA00000E915B00500110D8B42AD1C00E95157B
:1041EA00006E00C0A3FB0AD190CB00F091CB01F086
:1041FA00000E91BFFF0E026E036E0036009001366C
:10420A000236033600360090013602360336590E5E
:10421A000024F66E810E0120F76E000E0220F86E61
:10422A000900F5CF04F00900F5CF05F00900F5CF34
:10423A0006F00900F5CF07F09DCB00F09ECB01F008
:10424A009FCB02F0A0CB03F056EC06F00A0E046EE8
:10425A00000E056E066E076E56EC06F008C000F0FA
:10426A0009C001F00AC002F00BC003F0300E0024AE
:10427A00926FD3D095AB45D090CB00F091CB01F0A3
:10428A00000E91BFFF0E026E036E003600900136DB
:10429A000236033600360090013602360336170E10
:1042AA000024F66E820E0120F76E000E0220F86ED0
:1042BA000900F5CF04F00900F5CF05F00900F5CFA4
:1042CA0006F00900F5CF07F09DCB00F09ECB01F078
:1042DA009FCB02F0A0CB03F056EC06F00F0E0016AF
:1042EA00000E011602160316010E0024F66E840E45
:1042FA000120F76E000E0220F86E0900F5CF92FB3E
:10430A0044D090CB00F091CB01F0000E91BFFF0E8C
:10431A00026E036E0036009001360236033600360E
:10432A000090013602360336170E0024F66E820E0E
:10433A000120F76E000E0220F86E0900F5CF04F096
:10434A000900F5CF05F00900F5CF06F00900F5CF11
:10435A0007F09DCB00F09ECB01F09FCB02F0A0CBE3
:10436A0003F056EC06F00F0E0016000E01160216A8
:10437A000316120E0024F66E840E0120F76E000E4C
:10438A000220F86E0900F5CF92FB47D090CB00F0DF
:10439A0091CB01F0000E91BFFF0E026E036E003644
:1043AA000090013602360336003600900136023696
:1043BA0003361B0E0024F66E800E0120F76E000EE7
:1043CA000220F86E0900F5CF04F00900F5CF05F0D8
:1043DA000900F5CF06F00900F5CF07F09DCB00F0F4
:1043EA009ECB01F09FCB02F0A0CB03F056EC06F077
:1043FA00070E0014926F300E92270FD0A351000AB5
:10440A00D8B4F2D6A351C00AD8B4EED6A351800AC2
:10441A00D8B430D7A351400AB9E081CBE1FF82CBAF
:10442A00E2FF92CBE6FF814B822BA14BA22BCAD68D
:10443A0095A71AD0800E006E800E9419005C02E1D6
:10444A009351000811E281CBE1FF82CBE2FF200EFB
:10445A00E66E814B822BA14BA22B010E935F000EBD
:10446A00945B93519411EFE132EF12F0A1CB00F07B
:06447A00A2CB01F01200CC
:1044800081CB00F00032009E0032009E0032009E80
:104490000032009E82CBE1FF83CBE2FF300E00248E
:1044A000E66E010E0B018225E16E000E8321E26EA5
:1044B0000F0E8115006E300E002600C0E6FF020EC2
:0E44C0008225E16E000E8321E26EE66A120094
:1044CE007B0E0B017F6F0B0E806F76CB81FB77CB54
:1044DE0082FB78CB83FB79CB84FB7ACB85FB7F0E7B
:1044EE00866F0B0E876F2DEC12F000C07DFB01C0A6
:1044FE007EFB00507625E16E01507721E26EE66A72
:0A450E007DCB00F07ECB01F012001F
:10451800D8906E3766375E3656364E3646363E3655
:1045280036362E3626361E361636D8906F3767370B
:104538005F3657364F3647363F3637362F362736AB
:104548001F361736D8907037683760375836503668
:104558004836403638363036283620361836D89021
:1045680071376937613759365136493641363936E8
:104578003136293621361936D89072376A3762377C
:104588005A3652364A3642363A3632362A36223683
:104598001A36D89073376B3763375B3653364B36DA
:1045A80043363B3633362B3623361B36D890743792
:1045B8006C3764375C3654364C3644363C363436C1
:1045C8002C3624361C36D89075376D3765375D36EE
:1045D80055364D3645363D3635362D3625361D365B
:0245E8001200BF
:1045EA00020E0B01766F000E776FB1EC10F00B0123
:1045FA007A6B7B6B9D9A920E0A019025E16E0A0EE8
:10460A009121E26EE66A000E915D02E1160E905D5E
:10461A00D8B0BFD0000E006E9151005C02E19051FB
:10462A001308D8B0B6D0020E0B01786F000E796F5E
:10463A000A0191510B01795D04E10A0190510B01C4
:10464A00785D2FE2920E7825E96E0A0E7921EA6EDC
:10465A00EE503B0A23E1920E7825E16E0A0E79218B
:10466A00E26EE66ACF0E7A257E6F090E7B217F6F96
:10467A00920E7625816F0A0E7721826FB7EC11F0C0
:10468A007ECBE1FF7FCBE2FF00C0E6FF7A4B7B2BBC
:10469A00010E7825766F000E7921776F784B792B8A
:1046AA00C7D7D2C97CFB000E7D6FD4C9D2F9D3C952
:1046BA00D4F97CCBD3F9CFC9CAF9D0C9CBF9D1C9BE
:1046CA00C9F9D2C9C5F90901D25106080AE2C56B6E
:1046DA00370E0B01816F820E826F000E836FE3EC3F
:1046EA0010F0D3C9CCF9D4C905FA0B01816B826BDE
:1046FA00AAEC11F005CA81FB2EEC10F000C082FB77
:10470A00010E816FAAEC11F0CCC981FB2EEC10F0DE
:10471A0000C082FB020E816FAAEC11F0C5C981FBB1
:10472A002EEC10F000C082FB030E816FAAEC11F090
:10473A00CAC981FB2EEC10F000C082FB040E816F07
:10474A00AAEC11F0CBC981FB2EEC10F000C082FB61
:10475A00050E816FAAEC11F0C9C981FB2EEC10F08D
:10476A0000C082FB060E816FAAEC11F0070E0B0146
:10477A00816F100E826FAAEC11F0CF0E0B01816FC0
:10478A00820E826F000E836FE3EC10F0B1EC10F032
:10479A0012D0180E0B01816F7F0E826F000E836F8D
:1047AA00E3EC10F0850E0B01816F7D0E826F000E17
:0847BA00836FE3EC10F0120024
:1047C200060E0C6E300E0D6E0D2EFED70C2EFCD783
:0447D20000001200D1
:1047D6000B01766B776B160E786F000E796F766B22
:1047E600776B800E7719006E800E005C02E1080E72
:1047F600765DD8B0ABD07651010FA96F765178258A
:10480600E96E77517921EA6EEECFAAFB080E78257C
:10481600006E000E7921016E76510024E96E775103
:104826000120EA6EEECFABFB100E7825006E000E6F
:104836007921016E76510024E96E77510120EA6EE6
:10484600EECFACFB180E7825006E000E7921016EB6
:1048560076510024E96E77510120EA6EEECFADFB6A
:10486600200E7825006E000E7921016E7651002407
:10487600E96E77510120EA6EEECFAEFB280E782561
:10488600006E000E7921016E76510024E96E775193
:104896000120EA6EEECFAFFB300E7825006E000EDB
:1048A6007921016E76510024E96E77510120EA6E76
:1048B600EECFB0FB380E7825006E000E7921016E22
:1048C60076510024E96E77510120EA6EEECFB1FBF6
:1048D600400E7825006E000E7921016E7651002477
:1048E600E96E77510120EA6EEECFB2FB480E7825CD
:1048F600006E000E7921016E76510024E96E775123
:104906000120EA6EEECFB3FB500E7825006E000E46
:104916007921016E76510024E96E77510120EA6E05
:10492600EECFB4FB580E7825006E000E7921016E8D
:1049360076510024E96E77510120EA6EEECFB5FB81
:0E494600FCEC05F00B01764B772B4BD71200E3
:10495400160E0901686F000E696FF20E0001A96F4F
:104964000A0EAA6FB1EC10F00B01766B776B800E18
:104974007719006E800E005C02E1080E765DD8B0F7
:104984002CD1765109016825E96E0B017751090193
:104994006921EA6EEECF81FB4BEC11F000C081FB84
:1049A40001C082FB30EC11F0765109016825006EDC
:1049B4000B01775109016921016E080E0024E96E8B
:1049C400000E0120EA6EEECF81FB4BEC11F000C02B
:1049D40081FB01C082FB30EC11F07651090168259E
:1049E400006E0B01775109016921016E100E00243C
:1049F400E96E000E0120EA6EEECF81FB4BEC11F064
:104A040000C081FB01C082FB30EC11F0765109013A
:104A14006825006E0B01775109016921016E180E9A
:104A24000024E96E000E0120EA6EEECF81FB4BEC10
:104A340011F000C081FB01C082FB30EC11F0765113
:104A440009016825006E0B01775109016921016E86
:104A5400200E0024E96E000E0120EA6EEECF81FBE9
:104A64004BEC11F000C081FB01C082FB30EC11F073
:104A7400765109016825006E0B01775109016921FE
:104A8400016E280E0024E96E000E0120EA6EEECFBE
:104A940081FB4BEC11F000C081FB01C082FB30ECC8
:104AA40011F0765109016825006E0B017751090157
:104AB4006921016E300E0024E96E000E0120EA6EB9
:104AC400EECF81FB4BEC11F000C081FB01C082FBF7
:104AD40030EC11F0765109016825006E0B01775115
:104AE40009016921016E380E0024E96E000E0120CF
:104AF400EA6EEECF81FB4BEC11F000C081FB01C0EC
:104B040082FB30EC11F0765109016825006E0B012F
:104B1400775109016921016E400E0024E96E000EEF
:104B24000120EA6EEECF81FB4BEC11F000C081FB5B
:104B340001C082FB30EC11F0765109016825006E4A
:104B44000B01775109016921016E480E0024E96EB9
:104B5400000E0120EA6EEECF81FB4BEC11F000C099
:104B640081FB01C082FB30EC11F07651090168250C
:104B7400006E0B01775109016921016E500E00246A
:104B8400E96E000E0120EA6EEECF81FB4BEC11F0D2
:104B940000C081FB01C082FB30EC11F076510901A9
:104BA4006825006E0B01775109016921016E580EC9
:104BB4000024E96E000E0120EA6EEECF81FB4BEC7F
:104BC40011F000C081FB01C082FB30EC11F0B1ECAC
:0C4BD40010F00B01764B772BCAD61200B4
:104BE00078CB01F0010E006E015004E00036009019
:104BF000FF0FFBD700C07CFB001C0B017B6F7A6BA7
:104C000076CBE9FF77CBEAFF796B7951070824E38C
:104C10007B51EF16120EE9267B51EF1600EC10F0D7
:104C20007C51EF1200EC10F0120EE95E7C51EF1493
:104C3000006E0CE079CB01F0010E006E015004E033
:104C400000360090FF0FFBD700507A13F6EC0FF000
:0E4C5000F6EC0FF0792BD9D77ACB00F01200DA
:104C5E0078CB01F0010E006E015004E0003600909A
:104C6E00FF0FFBD700C07CFB001E00C07BFB76CB8A
:104C7E00E9FF77CBEAFF0050EF16120EE9260B0183
:104C8E007A6B7A51070816E37ACB00F079CB01F0F4
:104C9E00005004E00132019EFF0FFBD77B51EF164F
:104CAE0001A002D07C51EF1225EC11F07C51EF12D5
:104CBE007A2BE7D7120EE95EF6EC0FF0F6EC0FF05A
:024CCE001200D2
:104CD00076CB04F077CB05F004C002F005C003F0FA
:104CE000044A052A78CB00F079CB01F00B01784B10
:104CF000792B00C0E9FF01C0EAFF02C0E1FF03C059
:104D0000E2FFEECFE6FF02C0E9FF03C0EAFFEE528A
:0E4D100001E0E2D776CB00F077CB01F0120085
:104D1E000B017A6B050E7A5D0AE27A517825E16E07
:104D2E00000E7921E26E200EE66E7A2BF3D77A51C1
:104D3E007825E16E000E7921E26EE66A7A077A51E5
:104D4E0078257B6F000E79217C6F0A0E046E000EA3
:104D5E00056E76CB00F077CB01F0DBEC0FF008C0E0
:104D6E0000F009C001F0300E00267BCBE1FF7CCBBA
:104D7E00E2FF00C0E6FF0A0E046E000E056E76CB53
:104D8E0000F077CB01F0DBEC0FF000C076FB01C03A
:104D9E0077FB000E011802E1000E001801E102D0AF
:064DAE007A07CDD71200C8
:104DB4000B01816B55EC10F000C003FA010E0B01DE
:104DC400816F55EC10F000C005FA020E0B01816FE3
:104DD40055EC10F000C0CCF9030E0B01816F55ECBB
:104DE40010F000C0C5F90050060802E20901C56BC5
:104DF400040E0B01816F55EC10F000C0CAF9050ECA
:104E04000B01816F55EC10F000C0CBF9060E0B01BD
:0C4E1400816F55EC10F000C0C9F91200CD
:104E2000A6A202D00000FCD7A69C77CBAAFF76CB27
:104E3000A9FF78CBA8FFA69EA684F2CF00F0F29E31
:104E4000550EA76EAA0EA76EA68200BE02D0F29ED5
:104E500001D0F28EA694A1B802D00000FCD7A19890
:024E600012003E
:104E62008FEC0FF0D00E0B01A96F2AEC0FF0110E90
:104E72000B01A96F2AEC0FF047EC09F0D10E0B01E0
:104E8200A96F2AEC0FF0010E0B01A96F26EC0AF0B4
:104E920000C077FB0B01A96B26EC0AF000C078FB7F
:104EA20028EC0FF0200E0B01796F77AF0AD02D0E90
:104EB200796FFF0E771B785302E1772B01D078814F
:104EC20007D07751630804E2640E775F310E796F81
:104ED20079CBBAF9300E796F7751090804E2792B50
:104EE2000A0E775FF9D779CBBBF9300E7725090126
:104EF200BC6F2E0EBD6F300E0B01776F300E796FC7
:104F0200785310E078BD03D0350E776F0BD0320E98
:104F1200776F350E796F78A101D0787F78AF02D0A4
:104F2200370E776F77CBBEF979CBBFF97651000A8E
:104F320004E1B00E0901C06F03D00901920EC06FE7
:084F4200430EC16FC26B1200A7
:104F4A0078CB01F0010E006E015004E000360090AB
:104F5A00FF0FFBD700C07AFB001E76CBE9FF77CBA9
:104F6A00EAFF0050EF16120EE9260050EF1622EC67
:104F7A0012F00B017A51EF12120EE95E25EC11F0D4
:104F8A007A51EF14796F7951000A000ED8A4010EF4
:0C4F9A00796F22EC12F079CB00F01200CD
:104FA6000B017D6B77AF0DD0010E7D6F78CBE1FFE6
:104FB60079CBE2FF2D0EE66E761F771F764B772BA9
:104FC60007D07D6B78CBE1FF79CBE2FF200EE66E52
:104FD60076CB00F077CB01F001320032019E013230
:104FE6000032019E01320032019E01320032019EE2
:104FF60000C07AFB010E78257E6F000E79217F6F47
:105006000A0E046E25EC05F00A0E046E25EC05F07A
:1050160008C000F0300E00267ECBE1FF7FCBE2FF1A
:1050260000C0E6FF010E7825E96E000E7921EA6ED2
:10503600EE50300A08E1010E7825E16E000E792166
:10504600E26E200EE66E020E78257E6F000E792146
:105056007F6F0A0E046E7ACB00F025EC05F008C0CF
:1050660000F0300E00267ECBE1FF7FCBE2FF00C0D2
:10507600E6FF76CB7BFB77CB7CFB0F0E7615006EBF
:1050860077CB01F0000E011600C07BFB01C07CFB54
:10509600710E046E020E056EFEEC09F000C07BFB7D
:1050A60001C07CFB030E7825E16E000E7921E26ECD
:1050B6002E0EE66E040E78257E6F000E79217F6F28
:1050C600E80E046E030E056E7BCB00F07CCB01F080
:1050D600DBEC0FF0300E00267ECBE1FF7FCBE2FF4C
:1050E60000C0E6FF050E78257E6F000E79217F6FE2
:1050F600640E046E000E056E7BCB00F07CCB01F0D7
:10510600DBEC0FF00A0E046E000E056EDBEC0FF002
:1051160008C000F009C001F0300E00267ECBE1FF8A
:105126007FCBE2FF00C0E6FF060E7825E16E000E9B
:105136007921E26EE66A09011F6B206B0B017D5136
:10514600010A17E17ACB00F0000E016EE80E046E3C
:10515600030E056EFEEC09F07B5100240001796F09
:105166000B017C51012000017A6F000E7B6F7C6F72
:105176001AD07ACB00F0000E016EE80E046E030E14
:10518600056EFEEC09F00B017B5100267C510122D5
:10519600005000080001796F01C07AF0000E7A57BE
:0851A600000E7B6F7C6F12000C
:1051AE00F29EF20E0001A96F0A0EAA6FA851000A14
:1051BE00D8A40ED1B4C081FBB5C082FBAB0E0B01DF
:1051CE00836F000E846F080E856F000E866F6DEC78
:1051DE0010F0080E0001B425E16E000EB521E26E4E
:1051EE00200EE66EA9C081FBAAC082FB7F0E0B01CA
:1051FE00836F7C0E846F000E856F05EC10F0B4C0CB
:10520E0081FBB5C082FBAB0E0B01836F000E846F6A
:10521E00080E856F000E866F6DEC10F0080E000103
:10522E00B425E16E000EB521E26E200EE66EB6C01C
:10523E0081FBB7C082FB030E006E000E016EC5C966
:10524E0004F0000E056EFEEC09F0E30E0024E96E8C
:10525E00000E0120EA6EEECF83FBEECF84FBEECF85
:10526E0085FB05EC10F0050E0001B625E16E000E73
:10527E00B721E26E200EE66E060EB625E16E000E2A
:10528E00B721E26EFAC0E6FF070EB625E16E000EFC
:10529E00B721E26EFBC0E6FF080EB625E16E000EEA
:1052AE00B721E26E200EE66EF8C081FBF9C082FBDC
:1052BE00030E006E000E016EC4C904F0000E056EE2
:1052CE00FEEC09F0B80E0024E96E000E0120EA6E25
:1052DE00EECF83FBEECF84FBEECF85FB05EC10F01B
:1052EE00070E0001F825E16E000EF921E26E200E88
:1052FE00E66E080EF825E16E000EF921E26E320E12
:10530E00E66E090EF825E16E000EF921E26E300E02
:10531E00E66EE1C0E1FFE2C0E2FF00C1E6FF010E72
:10532E00E125E16E000EE221E26E01C1E6FFDFC073
:10533E0081FBE0C082FBBA0E0B01836F090E846FF6
:10534E00060E856F000E866F6DEC10F0060E0001D6
:10535E00DF25E16E000EE021E26E7F0EE66E070E97
:10536E00DF25E16E000EE021E26E430EE66E080EC2
:10537E00DF25E16E000EE021E26E200EE66E7EC0AD
:10538E0081FB7FC082FB6A0E0B01836F090E846F57
:10539E00060E856F000E866F6DEC10F0060E000186
:1053AE007E25E16E000E7F21E26E7F0EE66E070E09
:1053BE007E25E16E000E7F21E26E430EE66E080E34
:1053CE007E25E16E000E7F21E26E200EE66E5AD033
:1053DE00A9C081FBAAC082FBEC0E0B01836F820E6B
:1053EE00846F000E856F05EC10F0B4C081FBB5C064
:1053FE0082FBAB0E0B01836F000E846F080E856F60
:10540E00000E866F6DEC10F0080E0001B425E16EF3
:10541E00000EB521E26E200EE66E80C081FB81C0CB
:10542E0082FBFA0E0B01836F000E846F080E856FE0
:10543E00000E866F6DEC10F0080E00018025E16EF7
:10544E00000E8121E26E200EE66E090E8025E16EC1
:10545E00000E8121E26EE66A0901B36B090E0001AE
:10546E0080250B01816F000E000181210B01826FDF
:10547E00740E836F090E846F3F0E856F000E866F5C
:10548E006DEC10F05F0E0001A925E16E000EAA2151
:08549E00E26EE66AF28E1200D4
:1054A600680E0901F16F0A0EF26F000EF36F000E1F
:1054B600F46F1E0EED6F1F0EEE6F000EEF6F000EF7
:1054C600F06F8E0EDD6F120EDE6F000EDF6F000EB8
:1054D600E06F4C0ED96F140EDA6FA90EDB6F0B0E50
:1054E600DC6F540EE56F1E0EE66FA90EE76F0B0E0E
:1054F600E86F500EE16F1E0EE26F000EE36F000EB6
:10550600E46F949894968B988B9694889486C79E0D
:08551600C79C380EC66E12009E
:10551E000900F5CFE6FF0006FBE10106F9E11200F6
:10552E0076CB7AFB77CB7BFB7ACB81FB7BCB82FB7B
:10553E001BEC11F000C07CFB0B017A517825016E3B
:10554E007B517921026E7651015CE16E77510258E2
:10555E00E26E00C0E6FF7C51000A01E119D0020E96
:10556E000B6EA00E0C6E920E0D6E0D2EFED70C2E27
:10557E00FCD70B2EFAD700007A4B7B2B800E7B19B3
:10558E00006E800E030A005C02E1FF0E7A5DCCE332
:10559E007A517825006E7B517921016E7651005C2F
:0C55AE00E16E77510158E26EE66A1200CF
:1055BA007A0E0B01706F030E716FB70E726F0B0EBE
:1055CA00736FFF0E0A01EA6FFF0EEB6F000EEC6FAE
:1055DA00000EED6FFF0EE66FFF0EE76F000EE86F2D
:1055EA00000EE96FFF0EEE6FFF0EEF6F000EF06F09
:1055FA00000EF16FAC8A900EAB6E948E949C9EAAAC
:0A560A0003D0AECF00F0FBD7120072
:105614003F0E806E0F01386B2F0E926E9296929809
:105624008998546BFF0E816EFF0E936E396B9382D3
:10563400826A3A6B948E949C949A8B9A94909494E4
:1056440094928B808B928B94030E966E606A1200F8
:105654008FEC0FF0D00E0B01A96F2AEC0FF00B01A9
:10566400A96B2AEC0FF047EC09F0D10E0B01A96FDE
:105674002AEC0FF0010E0B01A96F26EC0AF000C012
:1056840003FA010E0B01A96F26EC0AF000C005FA1B
:10569400010E0B01A96F26EC0AF000C0CCF9010E33
:1056A4000B01A96F26EC0AF000C0C5F900500608EA
:1056B40002E20901C56B010E0B01A96F26EC0AF089
:1056C40000C0CAF9010E0B01A96F26EC0AF000C054
:1056D400CBF900C081FB06EC11F000C0C4F9A96B42
:1056E40026EC0AF000C0C9F928EC0FF0CCC981FB04
:1056F400AB0E0B01826F000E836F40EC22F03A0E6A
:105704000001AD6F05CA81FBAE0E0B01826F000E66
:10571400836F40EC22F03A0E0001B06F03CA81FBA4
:10572400B10E0B01826F000E836F40EC22F000017A
:10573400B36BCAC981FBFA0E0B01826F000E836F33
:1057440040EC22F02F0E0001FC6FCBC981FBFD0E53
:105754000B01826F000E836F40EC22F02F0E0001CC
:10576400FF6FC9C981FB000E0B01826F010E836FAD
:1057740040EC22F00101026B0B017651010A22E197
:10578400200EB76FBDEC01F0FA0E0B01816F000E15
:10579400826F30EC11F0040E816F850E826F000E63
:1057A400836FE3EC10F0AB0E0B01816F000E826F80
:1057B40030EC11F0040E816F850E826F000E836F42
:0657C400E3EC10F01200FE
:1057CA0076CB02F077CB03F002C000F003C001F001
:1057DA00024A032A00C0E9FF01C0EAFFEE5201E0D3
:1057EA00F3D70B017651025C006E77510358016EB4
:0A57FA00010E005E000E015A1200BD
:105804000A01906B916B000E915D02E1510E905D67
:1058140012E2920E9025E16E0A0E9121E26EE66A82
:10582400010E9025006E000E9121016E00C090FAC9
:1058340001C091FAE8D78E6B8F6B906B916B8B6B79
:105844008C6B8D6BAB98AB88F28CAECF8BFA9D8A48
:06585400E46BE56B12009D
:10585A0076CB04F077CB05F004C0E9FF05C0EAFF78
:10586A00EE5203E0044A052AF7D704C002F005C045
:10587A0003F0044A052A78CB00F079CB01F00B013A
:10588A00784B792B00C0E9FF01C0EAFF02C0E1FFB3
:10589A0003C0E2FFEECFE6FF02C0E9FF03C0EAFF62
:1058AA00EE5201E0E2D776CB00F077CB01F012009E
:1058BA00160E096E000E0A6E160E096E000E0A6E9C
:1058CA00056A066A056A066A800E0618006E800E68
:1058DA00005C02E10C0E055C4CE205500B017625DA
:1058EA00E96E06507721EA6EEECF01F0030E006EE4
:1058FA0001C007F0000E086E005005E00736079059
:10590A000836FF0FFAD7036A046A800E0418006E7D
:10591A00800E005C02E1080E035C28E203500724B3
:10592A00006E04500820016E110E0024E96E010E6B
:10593A000120EA6E030E026E05C000F006C001F0F7
:10594A00025005E0003600900136FF0FFAD70350E7
:10595A0000260450012200500924E16E01500A2059
:10596A00E26EEECFE6FF034A042ACFD7054A062A9B
:04597A00ABD7120095
:10597E00310ECD6ECD823C0ECF6EB00ECE6E9E90A1
:10598E009F800B016E6B6F6B6C6B6D6BCD909D90F2
:02599E001200F5
:1059A0003C0ECF6EB00ECE6E76CB6EFB77CB6FFB20
:0E59B0000B016C6B6D6BCD809E909D80120084
:1059BE00090E0B6E1E0E0C6EE40E0D6E0D2EFED726
:1059CE000C2EFCD70B2EFAD700000F0E0B01A96F71
:1059DE00AA6BAB6BAC6BAD6BAE6BAF6BB06BB16BF5
:1059EE00B26BB36BB46BB56BFCEC05F0090E0B012F
:1059FE00A96FAA6BAB6BAC6BAD6BAE6BAF6BB06BD9
:105A0E00B16BB26BB36BB46BB56BFCEC05F00A0EFD
:105A1E000B01A96F010EAA6F010EAB6F010EAC6FD9
:105A2E00010EAD6F010EAE6F010EAF6F010EB06FB6
:105A3E00010EB16F010EB26F010EB36F010EB46F96
:105A4E00010EB56FFCEC05F00B0E0B01A96F070EE6
:105A5E00AA6F070EAB6F070EAC6F070EAD6F070E7A
:105A6E00AE6F070EAF6F070EB06F070EB16F070E5A
:105A7E00B26F070EB36F070EB46F070EB56FFCEC67
:105A8E0005F00C0E0B01A96F010EAA6F010EAB6F84
:105A9E00010EAC6F010EAD6F010EAE6F010EAF6F4A
:105AAE00010EB06F010EB16F010EB26F010EB36F2A
:105ABE00010EB46F010EB56FFCEC05F0020E0B6E0D
:105ACE00A00E0C6E920E0D6E0D2EFED70C2EFCD768
:105ADE000B2EFAD70000BCEC10F0D00E0C6EC90ED7
:105AEE000D6E0D2EFED70C2EFCD7000000001200FE
:105AFE0084EC42F09B6A700ED36E9B8CD26A160EAB
:105B0E000901686F000E696F7EDD546B8B6A8B9A8C
:105B1E008B800A0E0001826F000E836F8998090137
:105B2E00B69FB781B886030EB06E400EAF6EAC84D2
:105B3E003DDD090E0B6E1E0E0C6EE40E0D6E0D2E5F
:105B4E00FED70C2EFCD70B2EFAD700000C0E0B0135
:105B5E00B76FBDEC01F0090E0B6E1E0E0C6EE40E4F
:105B6E000D6E0D2EFED70C2EFCD70B2EFAD7000085
:105B7E00B1EC10F00001866BF20EA96F0A0EAA6F3F
:105B8E000901B86BB96B000EB95D02E1770EB85D15
:105B9E000AE2F20EB825E16E0A0EB921E26EE66A4D
:105BAE00B84BB92BF0D7B86BB96B000EB95D02E1EB
:105BBE003F0EB85D0BE2740EB825E16E090EB921E9
:105BCE00E26E200EE66EB84BB92BEFD7B36BEE0E2E
:105BDE000B01816F830E826F000E836FE3EC10F06A
:105BEE000901B86BB96B000EB95D02E10A0EB85D22
:105BFE001CE2030E006E000E016EB8C904F0B9C9A6
:105C0E0005F0FEEC09F0870E0024E96E000E01206F
:105C1E00EA6EEECF81FBEECF82FBEECF83FBE3ECA1
:105C2E0010F00901B84BB92BDED7090E0B6E1E0E04
:105C3E000C6EE40E0D6E0D2EFED70C2EFCD70B2E19
:105C4E00FAD70000B1EC10F0F20E0001A96F0A0EA7
:105C5E00AA6F940E0B01816F820E826F000E836FFE
:105C6E00E3EC10F00B01766B776BA9C078FBAAC042
:105C7E0079FB56DC020E0B6EA00E0C6E920E0D6EA4
:105C8E000D2EFED70C2EFCD70B2EFAD70000A9C076
:105C9E0081FBAAC082FB30EC11F0B1EC10F0900E3B
:105CAE000B01766F000E776FA9C078FBAAC079FB47
:105CBE0037DCA9C081FBAAC082FB30EC11F0B1EC3D
:105CCE0010F0060E0001A925E16E000EAA21E26E6B
:105CDE00E66A040EA9250B01816F000E0001AA21B0
:105CEE000B01826FB7EC11F000C0B5F9090E00017F
:105CFE00A925E16E000EAA21E26EE66A070EA9251D
:105D0E000B01816F000E0001AA210B01826FB7EC0F
:105D1E0011F000C0B4F9A00E766F000E776FA9C017
:105D2E0078FBAAC079FB97EC2AF0A9C081FBAAC028
:105D3E0082FB30EC11F0B1EC10F0060E0001A9253B
:105D4E000B01816F000E0001AA210B01826FB7ECCF
:105D5E0011F000C082F001C083F0F20E0001A96FB5
:105D6E000A0EAA6F0901B86BB96B000EB95D02E19C
:105D7E00780EB85D0AE2F20EB825E16E0A0EB92170
:105D8E00E26EE66AB84BB92BF0D73A0E0B01816F73
:105D9E007E0E826F000E836FE3EC10F0A9C081FBC4
:105DAE00AAC082FB040E0B01836F7D0E846F000E62
:105DBE00856F05EC10F0A9C081FBAAC082FB30EC08
:105DCE0011F0B1EC10F0660E0B01816F7B0E826F3D
:105DDE00000E836FE3EC10F0080E0001A925B46FDE
:105DEE00000EAA21B56F110EA925006E000EAA2174
:105DFE00016E00C0B6F001C0B7F01A0EA925F86FFB
:105E0E00000EAA21F96F240EA925E16F000EAA211A
:105E1E00E26F2B0EA925DF6F000EAA21E06F380E60
:105E2E00A9257E6F000EAA217F6F00C080F001C0F1
:105E3E0081F0B1EC10F0B30E0B01816F830E826F07
:105E4E00000E836FE3EC10F0280EC86E53EC2AF0B0
:105E5E00240E0B01816F830E826F000E836FE3ECB5
:105E6E0010F00E0E0B01816F400E826FAAEC11F036
:105E7E0081A23ED0AA0E0B01816F7E0E826F000EA4
:105E8E00836FE3EC10F00B01816B500E826FAAEC66
:105E9E0011F0010E0B01816F590E826FAAEC11F0F9
:105EAE00020E0B01816F140E826FAAEC11F0030E1D
:105EBE000B01816F020E826FAAEC11F0040E0B0122
:105ECE00816F010E826FAAEC11F0050E0B01816F2E
:105EDE00090E826FAAEC11F0120E0B01816F2EECDF
:105EEE0010F000C082FB060E816FAAEC11F009D0F3
:105EFE009E0E0B01816F830E826F000E836FE3EC9B
:105F0E0010F0010E0B01766F2AEC2BF0B1EC10F0B5
:105F1E00570E0B01816F820E826F000E836FE3ECC2
:105F2E0010F00B01766B31EC27F0BA0E0B01816F7E
:105F3E00090E826F30EC11F0B1EC10F0520E0B6EB8
:105F4E002B0E0C6E000E0D6E0D2EFED70C2EFCD7EA
:105F5E000B2EFAD70000800E0B01766F0F0E776FA7
:105F6E00786BA5EC27F0800E766F0F0E776F786B3F
:105F7E00CC0E796F2FEC26F0800E766F0F0E776FAA
:105F8E00786B440E796F2FEC26F0E1EC23F0800E47
:105F9E00766F0F0E776F786BA5EC27F0800E766F0D
:105FAE000F0E776F786BCC0E796F2FEC26F0800E7C
:105FBE00766F0F0E776F786BBE0E796F2FEC26F023
:105FCE00800E766F0F0E776F786BF0EC25F000C0B9
:105FDE0084F0000E0001856F800E0B01766F0F0EA0
:105FEE00776F786BF0EC25F000C004F10101036BC4
:105FFE000001845101010327000185510101042391
:10600E00080E0B01816F830E826F000E836FE3EC1F
:10601E0010F003C176FB04C177FB6A0E0B01786F9B
:10602E00090E796FD3EC27F06A0E0B01816F090E02
:10603E00826F30EC11F0B1EC10F0D7EC28F0A9C063
:10604E0081FBAAC082FB30EC11F0B1EC10F0B1EC88
:10605E0010F0A90E0B01816F810E826F000E836FFF
:10606E00E3EC10F0F18C0901FE6BFF6BF292F288FB
:10607E00D10E0B01816F810E826F000E836FE3ECE8
:10608E0010F0D08E9F8A9E8AAB88F28CF28E090118
:10609E00FC6BFD6BE80E0B01816F7F0E826F000EA5
:1060AE00836FE3EC10F064DC140E766F000E776FE6
:1060BE0070DC240EAD6EB1EC10F0000E0B016D19FC
:1060CE0002E1000E6C1901E1F8D7230EAD6EB1ECB2
:1060DE0010F00901FC6BFD6BC50E0B01816F7D0E7F
:1060EE00826F000E836FE3EC10F0B20E0B01816F26
:1060FE00820E826F000E836FE3EC10F08B8058DC03
:10610E00760E816F820E826F000E836FE3EC10F0BD
:10611E00BCEC10F0B1EC10F08B80B1EC10F02F0E47
:10612E000B01816F810E826F000E836FE3EC10F016
:10613E00180E0B01816F090E826F310E836F840E64
:10614E00846F000E856F05EC10F0180E0B01766F44
:10615E00090E776F5DEC2CF0A30E0B6E570E0C6EC6
:10616E00020E0D6E0D2EFED70C2EFCD70B2EFAD76F
:10617E0000007B0E0B01816F800E826F000E836F0D
:10618E00E3EC10F0160E0901686F000E696F0A013C
:10619E00016B026B000E025D02E1080E015DD8B0CC
:1061AE00D2D00151010F0B01A96F0A010151090152
:1061BE006825E96E0A01025109016921EA6EEECFE6
:1061CE00AAFB080E6825006E000E6921016E0A01F9
:1061DE0001510024E96E02510120EA6EEECFABFBB5
:1061EE00100E09016825006E000E6921016E0A016C
:1061FE0001510024E96E02510120EA6EEECFACFB94
:10620E00180E09016825006E000E6921016E0A0143
:10621E0001510024E96E02510120EA6EEECFADFB72
:10622E00200E09016825006E000E6921016E0A011B
:10623E0001510024E96E02510120EA6EEECFAEFB51
:10624E00280E09016825006E000E6921016E0A01F3
:10625E0001510024E96E02510120EA6EEECFAFFB30
:10626E00300E09016825006E000E6921016E0A01CB
:10627E0001510024E96E02510120EA6EEECFB0FB0F
:10628E00380E09016825006E000E6921016E0A01A3
:10629E0001510024E96E02510120EA6EEECFB1FBEE
:1062AE00400E09016825006E000E6921016E0A017B
:1062BE0001510024E96E02510120EA6EEECFB2FBCD
:1062CE00480E09016825006E000E6921016E0A0153
:1062DE0001510024E96E02510120EA6EEECFB3FBAC
:1062EE00500E09016825006E000E6921016E0A012B
:1062FE0001510024E96E02510120EA6EEECFB4FB8B
:10630E00580E09016825006E000E6921016E0A0102
:10631E0001510024E96E02510120EA6EEECFB5FB69
:10632E00FCEC05F0090E0B6E1E0E0C6EE40E0D6EDF
:10633E000D2EFED70C2EFCD70B2EFAD700000A011D
:10634E00014B022B27D7B1EC10F0A30E0B6E570E9C
:10635E000C6E020E0D6E0D2EFED70C2EFCD70B2ED4
:10636E00FAD700000B01766B2AEC2BF00B01766B43
:10637E0031EC27F0B1EC10F04B0E0B01816F800E5B
:10638E00826F000E836FE3EC10F0BA0E0B01816F7B
:10639E00090E826F30EC11F0B1EC10F0F28E0A01A2
:1063AE00006B0901F86BF96BF66BF76BA9C00BF17B
:1063BE00AAC00CF10A01E46BE56B0901FA6BFB6BE9
:1063CE00A9C076FBAAC077FBE5EC2BF000C00DF15F
:1063DE0001C00EF1180E766F090E776F890E786F69
:1063EE00830E796F000E7A6F00C07BFB01C07CFBC1
:1063FE0067EC22F0180E816F090E826F30EC11F0EF
:10640E000BC176FB0CC177FB5DEC2CF05F0E01012E
:10641E000D6F000E0E6F590E0B01816F830E826F82
:10642E00000E836FE3EC10F00A01076B086B006B34
:10643E00800E0B01766F0F0E776F786BA5EC27F041
:10644E00800E766F0F0E776F786BCC0E796F2FEC08
:10645E0026F0800E766F0F0E776F786B440E796F85
:10646E002FEC26F0E1EC23F0800E766F0F0E776F97
:10647E00786BA5EC27F0800E766F0F0E776F786B2A
:10648E00CC0E796F2FEC26F0800E766F0F0E776F95
:10649E00786BBE0E796F2FEC26F0800E766F0F0E96
:1064AE00776F786BF0EC25F000C084F0000E0001E1
:1064BE00856F800E0B01766F0F0E776F786BF0EC99
:1064CE0025F000C003F0026A000184510224006E20
:1064DE0085510320016E00C003F101C004F100C01C
:1064EE0076FB01C077FB6A0E0B01786F090E796F90
:1064FE00D3EC27F002EC2CF00901B7A13ED0020E2E
:10650E000001A86F740E0B01816F090E826F450E8C
:10651E00836F7D0E846F000E856F05EC10F0740E88
:10652E000B01766F090E776FE5EC2BF0800E0118DC
:10653E00026E800E025C02E13F0E005C0BE2740EF6
:10654E00766F090E776F0F0E786F010E796F2DEC47
:10655E002CF0E5D7FA0E816F840E826F000E836FDA
:10656E00E3EC10F0740E0B01816F090E826F30ECAC
:10657E0011F0B1EC10F00901B791800E006E800E93
:10658E000A010819005C02E1075107083FE2076B98
:10659E00086B896B8A6B800E8A19006E800E005C08
:1065AE0002E10C0E895D1CE2090E8925E16E0A0ED0
:1065BE008A21E26E0901F85101010B25006E0901D5
:1065CE00F95101010C21016E0A0189510024E96E75
:1065DE008A510120EA6EEECFE6FF894B8A2BDBD77C
:1065EE000901F84BF92B800E006E800EF919005C34
:1065FE0002E1F8515F0802E2F86BF96B090E0B012C
:10660E00766F0A0E776F5DEC2CF00FD00901B6BFD6
:10661E0003D0EBEC23F009D0000E0901F91902E1C9
:10662E00000EF81902E1AAEC24F00901F85101015B
:10663E000B25036E0901F95101010C21046E080EA0
:10664E000001A925016E000EAA21026E0450021847
:10665E0002E10150031821E1000E0A01081902E1BE
:10666E00070E07191AE1080E0001A9250B01766F16
:10667E00000E0001AA210B01776F5DEC2CF0EBEC04
:10668E0023F04A0E0B6E0E0E0C6E190E0D6E0D2EA5
:10669E00FED70C2EFCD70B2EFAD78CEC22F00A016B
:1066AE00896B8A6B000183510A018A5D04E1000146
:1066BE0082510A01895D0CE2150E0C6EC60E0D6E2E
:1066CE000D2EFED70C2EFCD70000894B8A2BEAD755
:1066DE00074B082B000E8D1902E1010E8C19D8A460
:1066EE00D4EF37F0920EE46F0A0EE56FE4CAE9FFBD
:1066FE00E5CAEAFFEE50480A56E1030EE425E96EBC
:10670E00000EE521EA6EEE50700A4DE1720E0B019D
:10671E00816F830E826F000E836FE3EC10F0810E9B
:10672E000B01816F810E826F000E836FE3EC10F010
:10673E00D70E0B01816F800E826F000E836FE3EC1C
:10674E0010F0040E0B01816F810E826F000E836FAD
:10675E00E3EC10F0800E0B01816F7A0E826F000E4B
:10676E00836FE3EC10F0E20E0B01816F7E0E826FF1
:10677E00000E836FE3EC10F0CF0E0B01816F7A0EDB
:10678E00826F000E836FE3EC10F0310E0B01816F00
:10679E007A0E826F000E836FE3EC10F0B1EC10F006
:1067AE000A01E46BE56BE4CAE9FFE5CAEAFFEE50C5
:1067BE00550A3AE1140EE425E96E000EE521EA6E63
:1067CE00EE50230A31E1DB0E0B01816F830E826FD7
:1067DE00000E836FE3EC10F0920E0B01816F0A0E28
:1067EE00826F30EC11F0B1EC10F0F5EC22F0DAEC37
:1067FE0026F003CA81FB06EC11F000C004FA05CAAC
:10680E0081FB06EC11F000C006FACCC981FB06EC48
:10681E0011F000C0F5F9CBC981FB06EC11F000C0F8
:10682E00C4F90A01E46BE56BE4CAE9FFE5CAEAFFC5
:10683E00EE504D0AD8A477D0010EE425E96E000E75
:10684E00E521EA6EEE50730A6EE1020EE425E96E62
:10685E00000EE521EA6EEE50670A65E1030EE425AF
:10686E00E96E000EE521EA6EEE503D0A5CE1E30EA4
:10687E000B01816F840E826F000E836FE3EC10F0BC
:10688E000A01D56B740E0B01766F090E776F960E9B
:10689E00786F0A0E796F68EC26F0740E816F090E10
:1068AE00826F30EC11F0B1EC10F0740E0B01766FBC
:1068BE00090E776FE5EC2BF0800E026E800E01183C
:1068CE00025C02E1005008081EE2740E766F090E9B
:1068DE00776FE5EC2BF0800E0118026E800E025CD5
:1068EE0002E13F0E005C0BE2740E766F090E776FBD
:1068FE00050E786F010E796F2DEC2CF0E6D70A0E8F
:10690E000001A86F0DD0F60E0B01816F810E826F04
:10691E00000E836FE3EC10F00001A86B0901746B9D
:10692E000A01E46BE56BE4CAE9FFE5CAEAFFEE5043
:10693E00410A3FE1010EE425E96E000EE521EA6E03
:10694E00EE50660A36E1020EE425E96E000EE521F0
:10695E00EA6EEE50660A2DE1030EE425E96E000E96
:10696E00E521EA6EEE503D0A24E1F50E0B01816F32
:10697E00840E826F000E836FE3EC10F0920E0B010B
:10698E00816F0A0E826F30EC11F0B1EC10F0040E34
:10699E000A01E425E96E000EE521EA6EEE50310A99
:1069AE0003E10901B68F02D00901B69F0A01E46B1B
:1069BE00E56BE4CAE9FFE5CAEAFFEE50530AD8A434
:1069CE0031D1010EE425E96E000EE521EA6EEE509E
:1069DE00700AD8A427D1020EE425E96E000EE52137
:1069EE00EA6EEE50650AD8A41DD1030EE425E96EB9
:1069FE00000EE521EA6EEE50650AD8A413D1040EFE
:106A0E00E425E96E000EE521EA6EEE50640AD8A484
:106A1E0009D1050EE425E96E000EE521EA6EEE5071
:106A2E003D0AD8A4FFD0FF0E0B01816F840E826F3A
:106A3E00000E836FE3EC10F0920E0B01816F0A0EC5
:106A4E00826F30EC11F0B1EC10F0230E0B01816F60
:106A5E00840E826F000E836FE3EC10F082C076FB23
:106A6E0083C077FB180E0B01786F090E796F8FECD0
:106A7E0026F0180E816F090E826F30EC11F0B1EC1A
:106A8E0010F0060E0A01E425E96E000EE521EA6E0D
:106A9E00EECFA9FBF2EC09F000C074FB070E0A0161
:106AAE00E425E96E000EE521EA6EEECFA9FBF2ECCD
:106ABE0009F000507427756B000E752374CBCDF959
:106ACE0075CBCEF9060E0A01E425E96E000EE5211E
:106ADE00EA6E300EEE5C006E016A000E015A0A0E6E
:106AEE00046E000E056EFEEC09F0070EE425D96E5D
:106AFE00000EE521DA6EDE5000240901FC6F000E57
:106B0E000120FD6F300EFC5F000EFD5B000E0B01D1
:106B1E00751902E1020E7419D8A478D0000E09017D
:106B2E00FD5D02E1010EFC5D71E3000EFD5D02E113
:106B3E00630EFC5D6BE2FCC982F0FDC983F0A60E0C
:106B4E000B01766F000E776F0A0E046E000E056E47
:106B5E00FCC900F0FDC901F0DBEC0FF0300E002493
:106B6E00786F10EC27F0030E0B6E080E0C6E770E7E
:106B7E000D6E0D2EFED70C2EFCD70B2EFAD7A70EB0
:106B8E000B01766F000E776F0A0E046E000E056E07
:106B9E00FCC900F0FDC901F0DBEC0FF008C000F0FD
:106BAE0009C001F0300E0024786F10EC27F0030EB0
:106BBE000B6E080E0C6E770E0D6E0D2EFED70C2E74
:106BCE00FCD70B2EFAD7460E0B01816F840E826F07
:106BDE00000E836FE3EC10F0A00E0B01766F000E2B
:106BEE00776F180E786F090E796F97EC2AF0180EE2
:106BFE00816F090E826F30EC11F0180E816F090E45
:106C0E00826F30EC11F0B1EC10F009D0AA0E0B012E
:106C1E00816F800E826F000E836FE3EC10F00A011D
:106C2E00E46BE56BE4CAE9FFE5CAEAFFEE50500AF1
:106C3E00D8A4B1D1010EE425E96E000EE521EA6E6D
:106C4E00EE504C0AD8A4A7D1020EE425E96E000E30
:106C5E00E521EA6EEE504D0AD8A49DD1030EE4252F
:106C6E00E96E000EE521EA6EEE503D0AD8A493D1EE
:106C7E00920E0B01766F0A0E776FE5EC2BF0800EFD
:106C8E000118026E800E025C02E1090E005CD8A0B3
:106C9E0082D1BE0E816F840E826F000E836FE3EC85
:106CAE0010F0E4CA81FBE5CA82FB30EC11F0B1ECC6
:106CBE0010F0060E0A01E425E16E000EE521E26EEB
:106CCE00E66A090EE425E16E000EE521E26EE66A43
:106CDE004E0E0B01816F840E826F000E836FE3ECFC
:106CEE0010F0900E0B01766F000E776F180E786F06
:106CFE00090E796F97EC2AF0180E816F090E826FCC
:106D0E0030EC11F0040E0A01E425E96E000EE521C7
:106D1E00EA6EEECFA9FBF2EC09F000C074FB050E93
:106D2E000A01E425E96E000EE521EA6EEECFA9FB1D
:106D3E00F2EC09F000507427756B000E7523070EE8
:106D4E000A01E425E96E000EE521EA6EEECFA9FBFD
:106D5E00F2EC09F000507427000E7523080E0A019C
:106D6E00E425E96E000EE521EA6EEECFA9FBF2EC0A
:106D7E0009F000507427000E752374CBCDF975CB36
:106D8E00CEF9040E0A01E425E96E000EE521EA6E45
:106D9E00300EEE5C006E016A000E015A0A0E046E91
:106DAE00000E056EFEEC09F0050EE425D96E000E00
:106DBE00E521DA6EDE5000240901FC6F000E012081
:106DCE00FD6F300EFC5F000EFD5B070E0A01E42521
:106DDE00E96E000EE521EA6E300EEE5C006E016A81
:106DEE00000E015A0A0E046E000E056EFEEC09F03E
:106DFE00080EE425D96E000EE521DA6EDE50002471
:106E0E000901C76F000E0120C86F300EC75F000E5C
:106E1E00C85B000E0B01751902E1040E7419D8A49B
:106E2E00ACD0000E0901FD5D02E10F0EFC5DD8A095
:106E3E00A4D0000EFD5D02E1180EFC5DD8B09DD011
:106E4E00000E006EC851005C02E1C7510308D8B0B5
:106E5E0094D0000E006EC851005C02E1C7510B08C1
:106E6E00D8A08BD0FCC9B5F9040E0A01E425E96E51
:106E7E00000EE521EA6EEECF8BFA940E0B01766FC3
:106E8E00000E776F8BCA78FB10EC27F0050E0A0107
:106E9E00E425E96E000EE521EA6EEECF8BFA950E33
:106EAE000B01766F000E776F8BCA78FB10EC27F014
:106EBE00030E0B6E080E0C6E770E0D6E0D2EFED79A
:106ECE000C2EFCD70B2EFAD7C7C9B4F9070E0A0140
:106EDE00E425E96E000EE521EA6EEECF8BFA970EF1
:106EEE000B01766F000E776F8BCA78FB10EC27F0D4
:106EFE00030E0B6E080E0C6E770E0D6E0D2EFED75A
:106F0E000C2EFCD70B2EFAD7080E0A01E425E96EDB
:106F1E00000EE521EA6EEECF8BFA980E0B01766F1E
:106F2E00000E776F8BCA78FB10EC27F0030E0B6EFA
:106F3E00080E0C6E770E0D6E0D2EFED70C2EFCD796
:106F4E000B2EFAD73E0E0B01816F840E826F000E50
:106F5E00836FE3EC10F0900E0B01766F000E776FDF
:106F6E00180E786F090E796F97EC2AF0180E816F54
:106F7E00090E826F30EC11F009D00B01720E816F89
:106F8E007E0E826F000E836FE3EC10F0B1EC10F00A
:106F9E000A01E46BE56B02EC2CF0000E0901FF19FF
:106FAE0002E1000EFE19D8B483EF32F0FE6BFF6BD8
:106FBE000001A85100080CE2800E006E800E0A013E
:106FCE000819005C02E107510B0802E20001A80754
:106FDE000B01766B2AEC2BF00B01766B31EC27F064
:106FEE00F20E0001A96F0A0EAA6FD7EC28F0090164
:106FFE00B6BF12D0800E006E800E0A010819005C1A
:10700E0002E10751070808E2A9C081FBAAC082FB72
:10701E0030EC11F0B1EC10F00001866B300EAB5D70
:10702E00006E0A0E0002F3CF01F0300EAC5D006E62
:10703E000050012601C0C6F90901B451015C06E3F6
:10704E00B551C65D03E2010E0001866F000E090107
:10705E00C65D05E3B451C65D02E20001866B000118
:10706E008651000A12E10A0E0B01A96FAA6BAB6BD7
:10707E00AC6BAD6BAE6BAF6BB06BB16BB26BB36B2E
:10708E00B46BB56BFCEC05F01DD00A0E0B01A96FAD
:10709E00020EAA6F020EAB6F020EAC6F020EAD6F38
:1070AE00020EAE6F020EAF6F020EB06F020EB16F18
:1070BE00020EB26F020EB36F020EB46F020EB56FF8
:0C70CE00FCEC05F089781FEF32F0FFD7D2
:1085080010EE79F09F0E006E090E016EDA0EF66E0F
:0E851800700EF76E000EF86E8FEC2AF0120057
:0470DA0000000000B2
:0170DE0001B0
:0270DF000000AF
:0270E1000000AD
:0270E300640047
:0270E5000000A9
:0170E70000A8
:1070E8003F83007979001C7B00F77B00B07B0001AF
:1070F8007E00C88300C27C003C7C00B57F00DE793E
:017108000086
:017109000085
:02710A00F20A87
:09710C0030303A30303A303000E6
:02711500000078
:02711700000076
:107119005684009E8400A68400AE84008E84006696
:1071290084005E84007684007E84006E8400B684C8
:07713900009684008684002B
:0271400000004D
:0271420000004B
:10714400CB8400D18400C58400D78400EF8400E997
:057154008400DD840051
:02715900000034
:09715B0030302F30302F303000AD
:02716400000029
:02716600200007
:047168000000000023
:02716C00F20A25
:02716E0000001F
:027170002000FD
:1071720000000000000000007E81A581BD99817E93
:107182007EFFDBFFC3E7FF7E6CFEFEFE7C38100055
:1071920010387CFE7C381000383838FEFED61038A5
:1071A2001010387CFE7C10380000183C3C1800009F
:1071B200FFFFE7C3C3E7FFFF003C664242663C00B5
:1071C200FFC399BDBD99C3FF0F03057D84848478F5
:1071D2003C4242423C187E183F213F202060E0C0E2
:1071E2003F213F212367E6C018DB3CE7E73CDB1881
:1071F20080E0F8FEF8E08000020E3EFE3E0E020045
:10720200183C7E18187E3C182424242424002400D0
:107212007F929272121212003E6338444438CC7844
:10722200000000007E7E7E00183C7E187E3C18FF27
:1072320010387C5410101000101010547C381000BC
:1072420000180CFE0C180000003060FE60300000D8
:1072520000004040407E0000002466FF66240000DB
:107262000010387CFEFE000000FEFE7C381000009C
:1072720000000000000000001010101010001000AC
:10728200242424000000000024247E247E242400E0
:10729200183E403C027C180000626408102646003A
:1072A2003048305688887600101020000000000018
:1072B2001020404040201000201008080810200034
:1072C200004438FE384400000010107C101000000A
:1072D20000000000001010200000007E00000000EE
:1072E20000000000001010000002040810204000FE
:1072F2003C42464A52623C001030501010107C0052
:107302003C42020C30427E003C42021C02423C00E3
:1073120008182848FE081C007E407C0202423C00FD
:107322001C20407C42423C007E42040810101000A7
:107332003C42423C42423C003C42423E0204380053
:10734200001010000010100000101000001010209B
:10735200081020402010080000007E00007E00007F
:1073620010080402040810003C420204080008004D
:107372003C425E525E403C00182442427E42420041
:107382007C22223C22227C001C22404040221C0003
:1073920078242222222478007E22283828227E0085
:1073A2007E222838282070001C2240404E221E00D7
:1073B2004242427E42424200381010101010380001
:1073C2000E04040444443800622428302824630054
:1073D2007020202020227E00635549414141410016
:1073E20062524A46424242003C42424242423C00CF
:1073F2007C22223C202070003C4242424A3C030054
:107402007C22223C282472003C42403C02423C0046
:107412007F49080808081C004242424242423C009E
:107422004141414122140800414141494949360044
:1074320041221408142241004122140808081C00A9
:107442007F42040810217F0078404040404078008D
:107452008040201008040200780808080808780014
:10746200102844820000000000000000000000FF1D
:10747200101008000000000000003C023E423F00E5
:107482006020202E31312E0000003C4240423C0060
:107492000602023A46463B0000003C427E403C0067
:1074A2000C1210381010380000003D42423E027C9F
:1074B20060202C322222620010003010101038009E
:1074C200020006020242423C6020242830282600A4
:1074D2003010101010103800000076494949490058
:1074E20000005C624242420000003C4242423C00D8
:1074F20000006C32322C20700000364C4C34040EEA
:1075020000006C322220700000003E403C027C00F1
:1075120010107C1010120C000000424242463A0049
:107522000000414122140800000041494949360047
:10753200000044281028440000004242423E027CDF
:1075420000007C0810207C000C10106010100C0051
:107552001010100010101000300808060808300043
:10756200324C0000000000001C14141C000000003B
:107572003C4240423C0C023C0044004444443E0035
:107582000C003C427E403C003C4238043C443E00FD
:10759200420038043C443E00300038043C443E0083
:1075A2003C2424243C00000000003C40403C061CDB
:1075B2003C423C427E403C0042003C427E403C0019
:1075C20030003C427E403C002400180808081C00A1
:1075D2007C823010101038003000180808081C0097
:1075E200421824427E4242001818003C427E420069
:1075F2000C007C2038207C000000330C3F443B0010
:107602001F24447F444447001824003C42423C006B
:107612000042003C42423C002010003C42423C00FE
:107622001824004242423C002010004242423C00E8
:1076320000420042423E023C4218244242241800C8
:107642004200424242423C0008083E40403E080896
:107652001824207020427C0044287C107C101000EA
:10766200F84C78444F4445E61C12107C1010906090
:107672000C0038043C443E000C00180808081C00AA
:107682000408003C42423C000004084242423C00E2
:10769200324C007C42424200324C0062524A460066
:1076A2003C44443E007E000038444438007C0000E4
:1076B2001000102040423C000000007E40400000CC
:1076C2000000007E0202000042C448F629438C1FDB
:1076D20042C44AF62A5F8202001000101010100005
:1076E20000122448241200000048241224480000FA
:1076F200228822882288228855AA55AA55AA55AAE4
:10770200DB77DBEEDB77DBEE1010101010101010C1
:1077120010101010F01010101010F010F0101010C7
:1077220014141414F414141400000000FC1414149F
:107732000000F010F01010101414F404F4141414D7
:1077420014141414141414140000FC04F414141467
:107752001414F404FC00000014141414FC000000BF
:107762001010F010F000000000000000F0101010E7
:10777200101010101F00000010101010FF00000069
:1077820000000000FF101010101010101F10101039
:1077920000000000FF00000010101010FF10101079
:1077A20010101F101F101010141414141714141496
:1077B200141417101F00000000001F1017141414D7
:1077C2001414F700FF0000000000FF00F714141467
:1077D20014141710171414140000FF00FF00000007
:1077E2001414F700F71414141010FF00FF00000027
:1077F20014141414FF0000000000FF00FF1010100A
:1078020000000000FF141414141414141F000000CC
:1078120010101F101F00000000001F101F1010107A
:10782200000000001F14141414141414FF14141470
:107832001010FF10FF10101010101010F0000000B8
:10784200000000001F101010FFFFFFFFFFFFFFFFEF
:1078520000000000FFFFFFFFF0F0F0F0F0F0F0F0AA
:107862000F0F0F0F0F0F0F0FFFFFFFFF00000000A2
:107872000000314A444A3100003C427C427C404094
:10788200007E424040404000003F54141414140053
:107892007E42201820427E0000003E4848483000C8
:1078A200004444447A40408000334C0808080800F1
:1078B2007C1038444438107C1824427E422418003C
:1078C20018244242242466001C20183C42423C00F8
:1078D200006295899562000002043C4A523C408055
:1078E2000C10203C20100C003C424242424242001A
:1078F200007E007E007E000010107C1010007C00D4
:107902001008040810007E000810201008007E00F5
:107912000C12121010101010101010101090906015
:107922001818007E0018180000324C00324C00007B
:107932003048483000000000000000181800000025
:1079420000000000180000000F08080808C82818E6
:10795200784444444400000030481020780000007D
:1079620000003C3C3C3C0000000000000000000025
:07797200286E756C6C290002
:10797900204469726563746F7279203A20433A5CD6
:107989005F4D696B726F435C5F4D657350726F6ACF
:107999006574735F4D696B726F435C486F726C6F8E
:1079A90067655F31326D617472696365735F3878D9
:1079B900385F646566696C745F3936626974735FD0
:1079C90061736D5F31384632364B32325F3139314E
:0579D90032200D0A0040
:1079DE00205049432045656570726F6D203A2048EE
:1079EE006F726C6F67655F385F4D61747269636546
:1079FE003878385F646566696C5F446174655F48AA
:107A0E00657572655F31384632364B32325F3139C9
:107A1E00313230375F456570726F6D2E69686578EB
:037A2E000D0A003E
:107A310020657420616666696368616765204461D9
:107A41007465207265647569742065742070617352
:107A51002064652074656D706572617475726573FB
:107A61002070656E64616E74206C65204D736720B3
:0F7A7100416666696368E9203C43523E0D0A0096
:107A8000204166663D313D41666669636865205404
:107A900072616D6520656E2062696E616972652034
:107AA000737572207465726D696E616C2073696E96
:107AB0006F6E2C20204166663D3020737572204D1C
:0F7AC00061747269636573203C43523E0D0A0086
:107ACF00204D73673D782E2E2E7820646520382048
:107ADF00E0203430206361726163746572657320D6
:107AEF0041666669636865206C65206D65737361B7
:107AFF00676520782E2E2E782070656E64616E7407
:0D7B0F002031206D6E203C43523E0D0A00D7
:107B1C002050726F6A6574203A20486F726C6F67E0
:107B2C00655F31325F4D6174726963653878385FB7
:107B3C00646566696C656D656E745F39366269740F
:107B4C00735F31384632364B32325F313931323134
:0A7B5C00342E6D637070690D0A008D
:107B660020496E697420646573203720706F696ED2
:107B7600746575727320737572206C6573207061FD
:107B86007274696573205641524941424C455320EF
:107B96006465206C61207472616D6520E020616609
:0A7BA600666963686572200D0A002D
:107BB00020557361676520646520313220726567E6
:107BC0006973747265732064652036342062697449
:107BD0007320706F7572206C6520646563616C61E1
:107BE000676520E020676175636865202E2E656EED
:077BF0002041534D0D0A0076
:107BF70020536F75726365203A20486F726C6F6708
:107C0700655F646566696C5F31325F4D6174726987
:107C17006365735F3878385F3936626974735F31CB
:107C2700384632364B32325F5F3139313231342E9A
:057C370063200D0A00AE
:107C3C0020436F6E666967204F7363696C6C617467
:107C4C00657572203A2050494331384632366B32D2
:107C5C00325F464F53435F696E7465726E655F3178
:107C6C003678342D36344D485A2E63666773636804
:037C7C000D0A00EE
:107C7F00202020202020202048483A4D4D3A5353B1
:107C8F00204A6F757220206A6A204D6F6973202019
:107C9F0020204141414120496E743D2B58582E58A8
:107CAF0058B043204578743D2B58582E5858B04340
:037CBF0020200082
:107CC2002054696E795F5254435F445333323331E7
:107CD2005F666F725F4149325F313931322E6D63B7
:107CE2006C206574202A2E68202C466F6E74203A10
:107CF200205468696E5F53535F323031392E480D1C
:027D02000A0075
:107D0400202020202020202048483A4D4D3A53532B
:107D1400204A6F757220206A6A204D6F6973202093
:107D2400204141414120496E743D2B58582E5858EA
:107D3400B043204578743D2B58582E5858B04320F2
:017D4400003E
:107D450056657273696F6E2031342F31322F313998
:107D55002031384632364B3232205061756C664AD6
:107D6500756A6F204142434445464748494A4B4C52
:107D75004D4E4F505152535455565758595A20004D
:107D850020553A30333B31323B31393B31383B3387
:107D9500363B30322020706F757220303320646599
:107DA50063656D6272652032303139202031384883
:107DB50033362030323D4D617264690D0A0D0A007B
:107DC500204269742042616E6720536F66742053A8
:107DD500504920205243323D436C6B202C52433195
:107DE5003D446F757420205243303D4353202D3E52
:0C7DF500204D4178373231393A0D0A0038
:107E0100205465726D696E616C20706F75722064AB
:107E110069616C6F6775652065742056697375209B
:107E2100206465726F756C656D656E742070726F1C
:097E31006772616D6D650D0A00B8
:107E3A0020496E697469616C69736174696F6E2037
:107E4A005452414D452046495845206427416666AB
:107E5A00696368616765207375722038206D617483
:087E6A0072696365730D0A00E3
:107E72002042414420504C4D2076616C756573213F
:107E8200206D7573742062652066726F6D205B31A0
:107E9200352E2E203233205D20746F205B2034205B
:087EA2002E2E203131205D007D
:107EAA0020496E69742076616C657572732052542C
:107EBA004320706172206465666175742061752063
:107ECA0030312073657074203230313820E020312F
:087EDA0034483539200D0A007F
:107EE2002053656570643D787820207669746573E7
:107EF200736520646520646566696C656D656E7482
:107F020020787820646520303120E0203939203C07
:067F120043523E0D0A007F
:107F18000D0A2052617070656C20666F726D617415
:107F280020646520636465203A2022553B4A4A3B19
:107F38004D4D3B41413B48483B4D4D3B6A533B23EC
:057F480022200D0A00DB
:107F4D000000007FCDCC4C7B0AD723786F120375D0
:107F5D0017B75171ACC5276EBD37066B95BF566708
:107F6D0077CC2B645F700961FFE65B5D08E53C3CF7
:047F7D006042221B21
:107F81000000007F000020820000488500007A8800
:107F910000401C8C0050438F0024749280961896E8
:107FA10020BC3E99286B6E9CF90215A0EC782DC17E
:047FB100CAF249E2E5
:107FB5002044657669636573203A204D4158373210
:107FC50031392028636D73292C525443204453338F
:107FD5003233312C204F57532044533138423230FD
:037FE5000D0A0082
:107FE800205465737420696E74657272757074209C
:107FF80054696D657231202032302078203130305C
:10800800206D73656320736F697420327365632014
:038018000D0A004E
:10801B00010000000800000040000000000200000A
:10802B000010000000800000000004000000200091
:10803B0000000001000000080000004000000000EC
:10804B002054656D706572617475726520696E740C
:10805B0065726E6520445333323331206469726527
:10806B006374652066756E6374696F6E203A2000C9
:10807B00204166666963686167652042756666655F
:10808B007220646570756973203C4465706172740D
:0F809B003E203234206C6F6E677321200D0A0077
:1080AA00204241442053706565642076616C756591
:1080BA0021206D757374206265747765656E202062
:0D80CA00303120616E64203938200D0A002D
:1080D700206578656D706C6520706F7572203A3118
:1080E70034204D61692032303138203032284C75C8
:0D80F7006E6469292031354833360D0A00CA
:1081040020506C616765204C756D696E6F7369747E
:10811400E9204D696E696D616C6520504C4D3D31AF
:0B812400383A30363C43523E0D0A0052
:10812F0020696E69742041666669636861676520BE
:10813F0031322063617273203A3C3031323334353F
:0A814F003637383930313E0D0A0092
:10815900010000000A00000064000000E8030000BC
:1081690010270000A086010040420F008096980069
:0881790000E1F50500CA9A3B84
:1081810020525443205570646174653A20553B3147
:10819100343B30353B31383B31353B33363B303284
:0881A100233C43523E0D0A008D
:1081A90020496E697420496E746572727570742005
:1081B9005242302C2073796E6368726F2031487A8D
:0881C90020525443200D0A006E
:1081D10020496E697420496E7465727275707420DD
:1081E10054696D6572312020262055415254205228
:0581F10058200D0A00FA
:1081F600204D736720646F69742065747265203E34
:1082060038206574203C36332063617273210D0A71
:018216000067
:108217000100000010000000000100000010000035
:108227000000010000001000000000010000001025
:108237000D0A45727265757220737572204A6F75E3
:10824700722053656D61696E65206A53210D0A00BE
:108257002054656D706572617475726520696E74FE
:0F82670065726E6520445333323331203D200061
:1082760020436C656172203132204D6174726963EE
:0E8286006573204D415837323139200D0A0002
:1082940020526563757065726520706172616D65E9
:0E82A4007472657320456570726F6D0D0A006F
:1082B20020496E6974203132204D617472696365A0
:0D82C20073204D415837323139200D0A002C
:1082CF0045637269747572652064616E73204453DF
:0D82DF00333233312E2E2E204F4B0D0A006E
:1082EC00202020202020202048483A4D4D3A53533E
:0C82FC00204A4A2F4D4D2F414120200008
:108308002054656D702E4578746572726965757252
:0C8318002044533138423230203A20001B
:108324002041637469766520736F727469652053A4
:0B83340051573D31487A3A200D0A00F5
:10833F00204D696B726F6320372E362E3020313807
:0A834F004632364B3232200D0A0090
:108359002044656D6D617261676520646563616C58
:09836900616765203A200D0A004D
:108372000D0A2048656C70203A2048656C703C43B9
:07838200523E20200D0A000D
:10838900204C6F6E67205472616D65203D20253544
:0583990064200D0A0044
:10839E002052652D4C6563747572652052544320CE
:0583AE002D3E2020001F
:1083B30020496E697420525443204453333233317D
:0583C3003A200D0A0044
:1083C80020416C696D203D332E33565F6D696E69AF
:0383D8000D0A008B
:1083DB0020436465205254432055706461746520BA
:0383EB003A200035
:1083EE002050726573656E746174696F6E203A20E9
:0383FE000D0A0065
:1084010030313233343536373839414243444546C9
:01841100006A
:1084120030313233343536373839616263646566F8
:018422000059
:0E842300204F6C64207370656564203D20005E
:0D84310030313233343536373839303100D0
:08843E00204E6577203D20006F
:08844600204E6577203D200067
:08844E00204F6C64203D20006A
:088456006572726575722E005B
:08845E004A75696E2020200020
:088466004D6169202020200077
:08846E0053657074656D2E006A
:088476004A75696C6C65740025
:08847E00416F757420202000FD
:08848600446563656D622E0080
:08848E00417672696C202000A8
:088496004E6F76656D622E0049
:08849E004A616E766965720007
:0884A6004665767269657200FB
:0884AE004D61727320202000D3
:0884B6004F63746F62726500F0
:0784BE00204364653A200031
:0684C5004D6172646900C4
:0684CB0044696D616E00C2
:0684D1004C756E646900A9
:0684D7004D6572637200A6
:0684DD0053616D656400AF
:0684E300204D73673D000F
:0684E90056656E6472008E
:0684EF004A657564690096
:0584F5004364653D0039
:0584FA004D73673D0019
:0584FF004364653D002F
:0385040020200034
:020000040030CA
:0D000100381F3CFFBF81FF0FC00FE00F4014
:0200000400F00A
:1000000020486F726C6F67652038204D617472698B
:1000100063657320387838202050494331384632A0
:10002000364B32322020464F53432036344D487AE7
:100030002C2052544320445333323331202C20554A
:10004000415254312031393230302C382C4E2C3141
:100050000D0A00FFFFFFFFFFFFFFFFFFFFFFFFFF96
:100060002020202020202020202020202020202090
:100070002020202020202020202020202020202080
:10008000202020202020202020FFFFFFFFFFFFFF57
:10009000504C4D3D32313A30360D0A00FFFFFFFF24
:1000A00053706565643D31300D0A00FFFFFFFFFFAF
:1000B000FFFFFFFFFFFFFFFFFFFFFFFFFFFFFFFF50
:1000C000FFFFFFFFFFFFFFFFFFFFFFFFFFFFFFFF40
:1000D000FFFFFFFFFFFFFFFFFFFFFFFFFFFFFFFF30
:1000E000FFFFFFFFFFFFFFFFFFFFFFFFFFFFFFFF20
:1003E0007061756C666A756A6F2032303139200031
:1003F000FFFFFFFFFFFFFFFFFFFFFFFFFFFFFFFF0D
:00000001FF
